:106C5E00011900000501013C0200000301FA0400C5
:106C6E00FA0500030A0A5A0B001E0C00FA0D000367
:106C7E000E00040F0164100096120132130AFA146A
:106C8E00010215000217010A1801FA1905321A013C
:106C9E000A1B01FA1C05321FFFFF20FFFF23011EF6
:106CAE002400642A00FA2B00FA2C50782D003D2E79
:106CBE0000462F001E30006432507833000034320C
:106CCE00FA350164360164370150380A643C0064B9
:106CDE003E003C3F000140FFFF411450420A5A4320
:106CEE000AC84405324500B44600FA470178480206
:106CFE00034C00FA4EFFFF500505510596520A321D
:106D0E00530B46540A96560102570546580002592F
:106D1E000A465A32FA5B010A5C0A325E000A5F00CA
:106D2E00FE61FFFF64021C66000167FFFF6A0A3CFA
:106D3E006B00006C3296730000740000780132799B
:106D4E0001327EFFFF81FFFF84FFFF8500AF8600CB
:106D5E00018700FA8901088A00009900009D0A96B1
:106D6E009E00019FFFFFA0FFFFFAFAFA0000050147
:106D7E00013C0200000301FA0400FA0500030A0AAE
:106D8E005A0B001E0C00FA0D00030E00040F0164D6
:106D9E00100096120132130AFA14010215000017A0
:106DAE00010A1801FA1905321A010A1B01FA1C050B
:106DBE00321FFFFF20FFFF23011E2400642A00FA6A
:106DCE002B00FA2C50782D003D2E00462F001E3041
:106DDE0000643250783300003432FA3501643601E3
:106DEE0064370150380A643C00643E003C3F0001A9
:106DFE0040FFFF411450420A5A430AC84405324527
:106E0E0000B44600FA47013C4802024C00FA4EFF1D
:106E1E00FF500606510596520A32530B46540A96F7
:106E2E00560101570546580001590A465A32FA5B77
:106E3E00010A5C0A325E000A5F00FE61FFFF640316
:106E4E001C66000167FFFF6A0A3C6B00006C3296FD
:106E5E007300007400007801327901327EFFFF81E9
:106E6E00FFFF84FFFF85FFFF86FFFF87FFFF89017E
:106E7E00028A00009900009D0A969E00019FFFFF66
:106E8E00A0FFFFFAFAFA0065006F00790083008D0B
:106E9E00009700A100AC00B600C000CA00D400DE0E
:106EAE0000E800F200580060006800700078008072
:106EBE0000880090009800A000A800B000B800C1A3
:106ECE0000C800D000D800DF00E600EE00F600415A
:106EDE000047004D00530059005F0065006C0071C3
:106EEE000077007D00830089008F0095009B00A233
:106EFE0000A700AC00B200B900C000C500CA00D2A5
:0A6F0E0000D500DD00E100E700EF10
:103A390090006AE0D3940440149007DAE0FEA3E012
:103A4900FF906C60127051E493F59980129007DA37
:103A5900E0FEA3E0FF906D7A127051E493F599901E
:103A690007DAE0FEA3E0FF906C5EE493FC74019337
:103A7900FDEFB50507EEB50403754E009007DA12A0
:103A890070382275A71085F97485FA757E017F0053
:103A9900E57512702AE5742FFF50010E8E5B8F5C5D
:103AA90090001FE0FCA3E0FDEF2DFDEE3CFC8C5DDA
:103AB9008D5E22E55EF5FBE55DF5FCD29322E55EC0
:103AC900F5E9E55DF5EAD29422E55EF5EBE55DF50C
:103AD900ECD29122E55EF5EDE55DF5EED29222E5B7
:103AE9005EF5FDE55DF5FED28722AE5BAF5C74063F
:103AF9008E048F05FF12701A8C5D8D5EAE5BAF5C14
:103B090074068E048F05FF1270458C5B8D5CE55C35
:103B1900455B60137406C3955CFFE4955BFE8E5BA1
:103B29008F5C785D12707EE574A85DB80015D39539
:103B39005E4010E574C3955EFFE4955DFE8E5D8F72
:103B49005E8010E574243CC3955EFFE4955DFE8EAE
:103B59005D8F5EAE5DAF5E743B6F4E6006743C6F09
:103B69004E701AAE5DAF5E743B6F4E700575740191
:103B79008003757402755E3A755D00800375740083
:103B8900229000AAE0B40104C20E8002D20E900075
:103B9900ABE0B40104C20F8002D20F9000E8E075D7
:103BA900F0DCA4FFAEF0740A8E048F05FF12701AC0
:103BB9009007D0ECF0A3EDF0A20B401674038C062D
:103BC9008D0712702A74011200399007CEEEF0A306
:103BD900EFF07E017F009000A6E012702A9000E9C4
:103BE900E08E048F05FF12701A740AFF12701A8D85
:103BF900619000F2E075F0DCA4FFAEF0740A8E0467
:103C09008F05FF12701A9007D4ECF0A3EDF0900025
:103C1900F4E060139000F4E0F5F0741684FF7E0080
:103C2900EF9007E2F0800674649007E2F09000EAF2
:103C3900E090008FF0900134E0900079F09000C39B
:103C4900E090007BF09000ECE090007CF090009810
:103C5900E090007DF09000DEE090007EF090011E83
:103C6900E0900082F0900182E0900083F09001835F
:103C7900E0900084F0900184E0900085F0A231B3D7
:103C89004016900182E0700C900183E0700690016B
:103C990084E060028002C23174E390008EF09000EB
:103CA900D3E0B40B0874E390008EF0805A9000D3EF
:103CB900E0B419129000E9E0906E7F12008CE49351
:103CC90090008EF080419000D3E0B41E129000E97C
:103CD900E0906E9D12008CE49390008EF080289005
:103CE90000D3E0B428129000E9E0906EC712008C6E
:103CF900E49390008EF0800F9000D3E0B4460890D2
:103D090000CAE090008EF0900103E0FE9000D1E03F
:103D19006E600A9000D1E0900103F0D230900092D9
:103D2900E0FE9000D0E0B50627900094E0FE9000F8
:103D3900EEE0B5061B900093E0FE9000FCE0B506AE
:103D49000F900095E0FE9000A3E06E7003023E76AE
:103D590090006AE0C394055008740290011FF08036
:103D690006740890011FF09000A3E0B401067400E6
:103D7900900109F09000A3E0B4020674009000EEEF
:103D8900F09000A3E0B4030674009000FBF09000EB
:103D9900EEE0D394014014741A900121F07400905C
:103DA90006E4F074009006E5F0800C74009001219F
:103DB900F0741A9006E4F09000D0E0601474069054
:103DC90000B7F074009006E8F074009006E9F080FE
:103DD9000C74009000B7F074069006E8F09000D0DB
:103DE900E0B4021474079000B8F074009006ECF087
:103DF90074009006EDF0800C74009000B8F0740720
:103E09009006ECF09000FCE0B40114741B900122C0
:103E1900F074009006F4F074009006F5F0800C74CC
:103E290000900122F0741B9006F4F0D2309000D07B
:103E3900E0900092F09000FCE0900093F09000EE8A
:103E4900E0900094F09000A3E0900095F09000A31A
:103E5900E090007AF09000FCE090007FF09000D0B4
:103E6900E0900080F09000EEE0900081F090010673
:103E7900E0B4011790002B740FF0A374FFF09000C9
:103E89002DE4F0A3F07402900106F0900106E0B46D
:103E9900034190002DE0FEA3E0FF90002BE0FCA37E
:103EA900E0FD127076741012702A7408120039EF4E
:103EB90090008BF0EF700674FF90008BF074009007
:103EC9000106F090002CE090008CF090002BE0901F
:103ED900008DF0900097E0900053F0900053E0249B
:103EE9000C900054F0900053E02418900055F09085
:103EF9000053E02424900056F0900053E0243090C1
:103F09000057F0900054E0D3943C400B900054E0EB
:103F1900C3943C900054F0900055E0D3943C400B7E
:103F2900900055E0C3943C900055F0900056E0D3C2
:103F3900943C400B900056E0C3943C900056F0909E
:103F49000057E0D3943C400B900057E0C3943C9059
:103F59000057F090005DE4F0900053E0643B600787
:103F6900900053E0B43C20900053E0B43B06740247
:103F790090005DF0900053E0B43C0690005D740140
:103F8900F09000537401F090005EE4F0900054E06A
:103F9900643B6007900054E0B43C20900054E0B4C6
:103FA9003B06740290005EF0900054E0B43C069029
:103FB900005E7401F09000547401F090005FE4F029
:103FC900900055E0643B6007900055E0B43C2090B8
:103FD9000055E0B43B06740290005FF0900055E094
:103FE900B43C0690005F7401F09000557401F090A4
:103FF9000060E4F0900056E0643B6007900056E0F2
:10400900B43C20900056E0B43B067402900060F086
:10401900900056E0B43C069000607401F0900056A0
:104029007401F0900061E4F0900057E0643B600790
:10403900900057E0B43C20900057E0B43B0674026E
:10404900900061F0900057E0B43C06900061740163
:10405900F09000577401F0900097E0FE9000FAE0AC
:104069002E900063F09000D5E0B40173900063E0F6
:1040790075F00C84AFF07E00EF4E7006900063E09F
:1040890004F0900063E00475F00C84AFF07E00EF5B
:104099004E7006900063E014F0900058E0B43D06BD
:1040A9009000587401F0900063E0D3943C400B9069
:1040B9000063E0C3943C900063F0900063E0D39404
:1040C9001E400D900063E0C3941E900064F0800AC6
:1040D900900063E0241E900064F075521E804190A8
:1040E9000063E075F00C84AFF07E00EF4E7006902F
:1040F9000063E004F0900063E00475F00C84AFF015
:104109007E00EF4E7006900063E014F0900063E0CB
:1041190075F00C84AFF07E00EF900063F075520CDF
:104129009000DEE0B4020280030242149000DDE058
:10413900D3943C400D9000DDE0C3943C9000DDF049
:10414900D2309000DDE0900058F0900058E075F012
:104159000C84AFF07E00EF4E7006900058E004F03A
:10416900900058E00475F00C84AFF07E00EF4E70BB
:1041790006900058E014F0900058E0B43D06900015
:10418900587401F0900058E0240C900059F0900008
:1041990058E0241890005AF0900058E02424900028
:1041A9005BF0900058E0243090005CF0900059E0FA
:1041B900D3943C400B900059E0C3943C900059F0D3
:1041C90090005AE0D3943C400B90005AE0C3943CD1
:1041D90090005AF090005BE0D3943C400B90005B58
:1041E900E0C3943C90005BF090005CE0D3943C40C9
:1041F9000B90005CE0C3943C90005CF0C226C2279F
:10420900C228C229C22AD22B0243389000DDE0908D
:104219000058F0900058E075F00C84AFF07E00EF84
:104229004E7006900058E004F0900058E00475F0D4
:104239000C84AFF07E00EF4E7006900058E014F049
:10424900900058E0B479069000587401F090005835
:10425900E0D3943C400F900058E0C3943C90005840
:10426900F0D2268002C226900058E0241890005906
:10427900F0900058E0243090005AF0900058E02463
:104289004890005BF0900058E0246090005CF0A238
:10429900269227A2269228A2269229A226922A901D
:1042A9000059E0D3943C4010900059E0C3943C90ED
:1042B9000059F0A226B3922790005AE0D3943C40CB
:1042C9001090005AE0C3943C90005AF0A226B39291
:1042D9002890005BE0D3943C402690005BE0D394A7
:1042E90078400D90005BE0C3947890005BF08010FB
:1042F90090005BE0C3943C90005BF0A226B3922946
:1043090090005CE0D3943C402690005CE0D3947824
:10431900400D90005CE0C3947890005CF0801090B0
:10432900005CE0C3943C90005CF0A226B3922A2280
:10433900C293C294C291C292C287C290E5B554EFAA
:10434900F5B5E5B554DFF5B5C296C295C2A0C297D9
:10435900C2A2C2A1E5B554BFF5B5E5B5547FF5B51F
:10436900E5B554FBF5B5C210755F469000E0E07005
:1043790005756E028003756E0375560075550090BC
:10438900001474FFF0A374DCF0C218C21AC21CC274
:104399001EC22074C890003FF074C8900043F074A6
:1043A900C8900047F074C890004BF074C890004F53
:1043B900F0755400755300C20B754700E570B409D8
:1043C90003757000756400900021E4F0A3F0757125
:1043D90010C213C214C215C216C2179007D0E0FE4C
:1043E900A3E0FF740312702A74011200399007CEFA
:1043F900EEF0A3EFF0C2027558007557009000184F
:10440900E4F0A3F0C232755A007559009000A2E099
:1044190075F032A4FDACF0900029ECF0A3EDF0C2E8
:1044290042A236B39205A237B39206A238B39207D5
:10443900A239B39208A23AB39209A23BB3920A22D3
:1044490075A71085F97485FA757E017F00E57512E7
:10445900702AE5742FFF50010E8E5B8F5CAC5DAD49
:104469005EEF2DFDEE3CFC8C5D8D5E123ABC123A7E
:10447900C7123AD2123ADD123AE875A7002285F935
:104489007485FA757E017F00E57512702AE5742F2F
:10449900FF50010E8E5B8F5C7E017F7690011BE0E1
:1044A90012702AAC5BAD5CED2FFFEC3EFE8E5D8F8A
:1044B9005EE55EF5EDE55DF5EE90008FE4F07412D2
:1044C900900066F02285F97485FA757E017F00E512
:1044D9007512702AE5742FFF50010E8E5B8F5C9068
:1044E90007D0E0FCA3E0FDEF2DFDEE3CFC8C5D8DDB
:1044F9005EE55EF5FDE55DF5FE22056522A2DBB30D
:1045090040089000EAE090008FF0A2DCB3400AC2B4
:1045190096C295C2A0C297C2A275D8402285A77338
:1045290075A710A2D8B34002C293A2D9B34002C260
:1045390094A2DAB34002C291A2DBB34002C292A2B2
:10454900DCB34002C28775D8408573A72290004723
:10455900E4936406600280FE74C89007D6F8E4F01C
:10456900E8A3F075B50075840175A70075FFA090E3
:104579000062E4F075C91075A70F75A1C775A7008A
:1045890075D90075CE0C75A70F75F1FE75F2FF751B
:10459900F30775F47875A4BA75A5FF75A60775AE06
:1045A9000075AFFF75D48175D5FF75D6FF75D7FF37
:1045B90075A70075A20175A14775F80975D8007529
:1045C900D90475DD0975DE0975D84075A71075D848
:1045D9000075D90475DA0975DB0975DC0975DD091A
:1045E90075DE0975D84075A70075E60875E7107579
:1045F900BC0175BE0475BD6C75BE0775BDA075BEE1
:104609000875BD0175BC0075BB1875BC2075BA0865
:1046190075E88075D11375A70F75E10575E2007509
:10462900C740124339759700759780740A12700A4A
:104639007597C0E5975420700280F8758F0275A7A9
:1046490000D2AF75980075A90C75A70F75AB4375A6
:10465900ADFB75AC1E75A71075C91875CA0075CB69
:104669000075C80475A700758912758E04758C00CC
:10467900758A00C2A9D28C758D00758B00D2ABD218
:104689008E75EF0675D944C2997509C87508001267
:1046990000E975B5001204E974639007D6F8E4F0EF
:1046A900E8A3F012037574C89007D6F8E4F0E8A3FC
:1046B900F07509647508001200E990007AE090002D
:1046C900A3F09000A3E0D39403400C74009000A3DE
:1046D900F0740090007AF0C2249000A3E090686919
:1046E900F82828738028A2B44002D224802075A714
:1046F9000F75F30F75A700A2A34002D224800F758E
:0E470900A70F75F31775A700A2A44002D224D3
:0C6869000246ED0246EF0246F702470827
:10471700A224B3405E757408E574D3940E501FE568
:10472700749007D6F8E4F0E8A3F012024475096420
:104737007508001200E97874740126F650DA7402DD
:104747009000DFF090007AE09000A3F09000A3E0E3
:10475700906875F828287380167400900109F08016
:0F4767000E74009000EEF0800674009000FBF0DE
:0C68750002475E0247600247680247705D
:10477600D223805C757401E574D39407501FE574E9
:104786009007D6F8E4F0E8A3F012024475096475C0
:1047960008001200E97874740126F650DA74019064
:1047A60000DFF090007AE09000A3F09000A3E09084
:1047B6006881F828287380167400900109F0800E2D
:0E47C60074009000EEF0800674009000FBF08E
:0C6881000247BC0247BE0247C60247CED9
:1047D400C223900079E0900134F090007AE09000D8
:1047E400A3F090007BE09000C3F090007CE0900088
:1047F400ECF090007DE0900098F090007EE0900056
:10480400DEF090007FE09000FCF0900080E09000EB
:10481400D0F0900081E09000EEF0900082E09001F2
:104824001EF0900083E0900182F0900084E09001FB
:1048340083F0900085E0900184F0900182E0700C98
:10484400900183E07006900184E060028004C2312C
:104854008002D2319000E9E07006740A9000E9F019
:104864009000CAE0700674E39000CAF09000D0E0B3
:1048740004900092F09000D1E0900103F0123B8A82
:10488400E5B54401F5B57406900068F07401900034
:1048940069F0740390006BF0740590006CF0741D63
:1048A40090006DF0740590006EF090006AE0B4041E
:1048B40006740490006EF0740190006FF074009020
:1048C4000074F07400900077F074FF900078F07436
:1048D4003690016DF0743090016EF0742D90016F7C
:1048E400F07432900170F07420900171F07435907E
:1048F4000172F07443900173F07479900174F07450
:104904006C900175F07420900176F074209001771A
:10491400F07420900178F07420900179F074209064
:10492400017AF0742090017BF0900105E090008BF7
:10493400F09000BCE090008CF09000BDE090008D01
:10494400F0A2B6B3920CA2B3B3920DA2A4B3922D6B
:10495400A2B4B3922EA2A3B3922F900087E4F07571
:104964007000743A900796F074FD900797F09000E9
:1049740088E4F09007D0E0FEA3E0FF740312702AED
:1049840074011200399007CEEEF0A3EFF0756F01B9
:10499400900066E4F0C22C756400C211D212C20207
:1049A400757200C234D203C235D204C236D205C2F3
:1049B40037D206C238D207C239D208C23AD209C2A3
:1049C4003BD20AC225C22BC23012009E756000750C
:1049D4006C007562007566327567007568007569EC
:1049E40000756A00756B00900021E4F0A3F0756D0A
:1049F40000D2B2D2A4D2B0D2B1D2A3D2A7D2A6D27C
:104A0400A5D2B79000A2E0D394FA400674FA9000BD
:104A1400A2F07E017F0090008DE012702A90008C3D
:104A2400E02FFF50010E90002BEEF0A3EFF0EFD338
:104A340094FFEE940F400790002BE4F0A3F0900055
:104A44008BE0700674FF90008BF09000DFE0D3944D
:104A540002400674019000DFF09000E0E0700575FC
:104A64006E028003756E039000E1E0D3940140066A
:104A740074009000E1F09000E7E0C3940A500674DB
:104A84000A9000E7F09000F1E0700674019000F1E4
:104A9400F09000F1E0B4FF0674FE9000F1F0900095
:104AA400F8E0D394FE400674FE9000F8F090011EE6
:104AB400E0D394024006740190011EF0900134E0AA
:104AC400D3940140067401900134F074019000FE07
:104AD400F074019000FFF07400900106F0740090EF
:104AE4000126F074299006DCF0742A9006E0F07434
:104AF400089006F0F0741C9006F8F0D29C9000D157
:104B0400E0D39404400674049000D1F0E571D3948A
:104B14001040037571109006DDE0D3940C400674C8
:104B2400009006DDF09006E1E0D3940C400674009A
:104B34009006E1F09006E5E0D3940C4006740090F2
:104B440006E5F09006E9E0D3940C40067400900664
:104B5400E9F09006EDE0D3940C400674009006ED65
:104B6400F09006F1E0D3940C400674009006F1F046
:104B74009006F5E0D3940C400674009006F5F0908E
:104B840006F9E0D3940C400674009006F9F0D2ECD8
:104B940075CF01A298B34005C298120646E54E604F
:104BA40006A299B3B340028005C299120C57E54F8F
:104BB40064016005E54FB4040280D5C28E7E107F87
:104BC40000E56512702AE58D75F010A4FDACF0EFD8
:104BD4002DFDEE3CFCE58B75F01084FF7E00ED2F7F
:104BE400FFEC3EFE8E558F56D28E9000C3E06009D6
:104BF4009000C3E0C3943D4002805690002312709D
:104C040038900023E0FEA3E0FF900025E0FCA3E041
:104C1400FDEFB5053CEEB50438B222A20BB3401348
:104C2400A222B34008E5B54404F5B58006E5B554C1
:104C3400FBF5B5900025E0FEA3E0FF900027E0FC23
:104C4400A3E0FDEF2DFDEE3CFC900025ECF0A3ED80
:104C5400F09000D0E060099000D0E0C394034002DB
:104C6400807D122D96A20BB35009900087E0C39467
:104C74002B400280069000BAE0F546E54675F00543
:104C8400A4FFAEF09007D8EEF0A3EFF09000A7E0F9
:104C9400C395624007E560C3956150079007D8E467
:104CA400F0A3F0AE2FAF309007D8E0FCA3E0FDEF07
:104CB400D39DEE9C4004C290800B900087E0C39487
:104CC400415002D2909000D0E0B40213A290B340BD
:104CD40008E5B554EFF5B58006E5B54410F5B59093
:104CE40000D0E0B4031C122EB1AE2FAF309007D821
:104CF400E0FCA3E0FDEFD39DEE9C4004D290800243
:104D0400C2909000ABE06009A2B3300D01B3B34090
:104D1400028039A2B3300D01B34031A2B3300F0188
:104D2400B3401C9000DEE0B40306A225B3B34002F6
:104D340080067404900066F0D225A20FB3920DA2EF
:104D44000FB330B301B34004A20F920DA2B6300CDE
:104D540001B350030253EEA2B6300C01B350030268
:104D640053EEA2B6300E01B3500302524E756F00DB
:104D74009000C3E0B43D13A20EB34008E5B554FB64
:104D8400F5B58006E5B54404F5B5055FA210B3B3E7
:104D94005013AE55AF56900014E0FCA3E0FDEDC3F4
:104DA4009FEC9E4003024F06E56EB4032EA232B37D
:104DB4004022E55FB43B03756E01E55FC3943B504D
:104DC400069000667401F0E55FD3943B40067402DC
:104DD400900066F0755F01D2328060E56EB4020621
:104DE400756E01755F3BE55FB43B05755F01804BF4
:104DF400900066E07036E55FC3943B500690006611
:104E04007401F0E55FD3943B40067402900066F0B1
:104E1400E55FC3943B5002D22CE55FD3943B400240
:104E2400D22CC296C295C2A0C297C2A29000E0E062
:104E3400B401051243398003755F01AE57AF58AC16
:104E440055AD56EF2DFDEE3CFC74028C068D071219
:104E540000398E578F589000C3E060099000C3E07A
:104E6400C3943D40028043900023E0FEA3E0FF9002
:104E740000C3E08E048F05FF12701A74018C068D36
:104E840007120039900027EEF0A3EFF0900027E01E
:104E9400F8A3E0900025C8F0A3C8F0900023E4F044
:104EA400A3F0C222E5B554FBF5B5A2B4B34002C2E7
:104EB4002EA2A4B34002C22DA2A3B34002C22FA2C9
:104EC4002CB34002C22C9000DEE0B40331A225B31F
:104ED4004006A226922B8002B22B9000ABE0601217
:104EE400E56E700EA225B35009A22B302601B3B390
:104EF400400280067405900066F0C2258002D22B21
:104F0400803AAE57AF58AC55AD56EF2DFDEE3CFC94
:104F140074018C068D071200398E578F58E56EC3C5
:104F24009402500DAC55AD5674B8C39D740B9C409F
:104F34000280091243397406900066F0E55FB43BC1
:104F4400127403900066F0D22C9000E0E0B40103E8
:104F5400124339AE59AF5AAC55AD56EF2DFDEE3C68
:104F6400FC8C598D5AAE55AF56EFD39DEE9C401133
:104F740090001BE0FAA3E0FBEBC394E8EA9403403F
:104F840002800690001B127038900018E0FEA3E027
:104F9400FFAC55AD56EF2DFDEE3CFC900018ECF047
:104FA400A3EDF09000E0E0B40118AE55AF567405DF
:104FB40012702A7401120039900014EEF0A3EFF07D
:104FC4008011AE55AF56740212702A900014EEF0A0
:104FD400A3EFF0C28E758D00758B00756500755654
:104FE40001755500D28EE55F240E75F00F84AFF085
:104FF4007E00EF4E7075900018E0F8A3E090001664
:10500400C8F0A3C8F0900016E0FEA3E0FFEF4E60E6
:105014000B7C7D7D69126F188E538F54900018E4B9
:10502400F0A3F0AE53AF547428BE00039F5010E5B4
:10503400642FFF50010E74011200398E538F548572
:1050440054649000E7E0A853B8000DD39554400889
:10505400E554900065F080099000E7E01490006545
:10506400F0E56E6006755400755300E55F640B60EF
:1050740005E55FB429099000D0E060031223D290C3
:1050840000D5E0B40114900063E0655F6007900010
:1050940064E0B55F03757000801E900063E0655F97
:1050A4006013900063E02418655F6009900063E07A
:1050B4002424B55F03757000A211B35006A210B387
:1050C400B3400302516F90009CE0B4017390011E41
:1050D400E0B40214120E26900090E075F0BEA4FF16
:1050E400AEF08E5D8F5E8056E56875F00A84FF7EB3
:1050F40000900596127051E0F55C755B00AE5BAFF5
:105104005C9000C1E012702A74648E048F05FF1253
:10511400701A8C5D8D5EE55E90001AF0AE5BAF5C3C
:1051240090009AE012702A74648E048F05FF127046
:105134001A74BE8C068D0712702A8E5D8F5E8017DE
:1051440090009AE075F0BEA4FFAEF08E5D8F5E9085
:1051540000C1E090001AF0E562C394CC5006E55E0D
:10516400455D70028003124449D211E56EB4010614
:10517400E55F641160028009757101900067740134
:10518400F0E56E60030252499000E3E0600D900088
:105194008FE0A853B800069554400280509000E375
:1051A400E0B4022F900053E0655F601F900054E06C
:1051B400655F6017900055E0655F600F900056E0F2
:1051C400655F6007900057E0B55F03757103756D07
:1051D40000800CC200756D00900021E4F0A3F090F3
:1051E400008FE060067409900066F08058900053C8
:1051F400E0B55F0B7571019000677401F080469013
:105204000054E0B55F0B7571017402900067F08083
:1052140034900055E0B55F0B75710174039000671D
:10522400F08022900056E0B55F0B75710174049014
:105234000067F08010900057E0B55F097571017444
:1052440005900067F0A20EB3920CA20EB330B60123
:10525400B350030253EE756F019000C3E0B43D13E5
:10526400A20EB34008E5B54404F5B58006E5B5548F
:10527400FBF5B5E5B54401F5B5742B900087F0A2B4
:105284000E920CE55FD3944A4014D210E55FD39498
:1052940085400B7404900066F0D22C755F46900034
:1052A400EBE0B40107E56BC3941440028009124398
:1052B400397413900066F0A234300301B35017A27E
:1052C40034B34008E5B54408F5B58006E5B554F7B0
:1052D400F5B5A2349203A235300401B35017A235B8
:1052E400B34008E5B54402F5B58006E5B554FDF5CF
:1052F400B5A2359204A236300501B3500FA236B3DD
:105304004004D2A18002C2A1A2369205A23730067F
:1053140001B3500FA237B34004D2908002C290A2CE
:10532400379206A238300701B35017A238B34008A9
:10533400E5B54410F5B58006E5B554EFF5B5A238EA
:105344009207A239300801B35017A239B34008E5D7
:10535400B54420F5B58006E5B554DFF5B5A239921C
:1053640008A23A300901B35017A23AB34008E5B590
:105374004440F5B58006E5B554BFF5B5A23A9209A7
:10538400A23B300A01B35017A23BB34008E5B54431
:1053940080F5B58006E5B5547FF5B5A23B920AE5E4
:1053A4006BC394415009740E900066F01243399017
:1053B400006EE0FE90006AE004C39E400990006A1B
:1053C400E0D39408400974FB900066F012433990CE
:1053D4000073E06015900073E0FE90006DE06E6075
:1053E4000974FE900066F0124339A22CB3400AC23D
:1053F40096C295C2A0C297C2A290011BE0600CAEF7
:1054040053AF547414BE00059F400280489000A31B
:10541400E090688DF8282873803BA2B4B35005A2AD
:105424002EB340028005124487D22E8028A2A3B353
:105434005005A22FB340028005124487D22F801555
:10544400A2A4B35005A22DB340028005124487D212
:055454002D8002800024
:10688D0002541C02541E0254310254440254570245
:02689D0054594C
:10545900A213B3B35008900058E0655F600280441E
:10546900A226302B01B340028030A201B35006A21C
:1054790000B3B340028023123A8C123ABC9000FC6C
:10548900E0B40113A202B34008E5B54440F5B58084
:1054990006E5B554BFF5B575A700C213D214D215E8
:1054A900D216D217A214B3B35008900059E0655F21
:1054B90060028044A227302B01B340028030A20150
:1054C900B35006A200B3B340028023123A8C123AB9
:1054D900C79000FCE0B40113A202B34008E5B5444B
:1054E90040F5B58006E5B554BFF5B575A700D213EB
:1054F900C214D215D216D217A215B3B35008900010
:105509005AE0655F60028044A228302B01B3400253
:105519008030A201B35006A200B3B3400280231227
:105529003A8C123AD29000FCE0B40113A202B340C3
:1055390008E5B54440F5B58006E5B554BFF5B57540
:10554900A700D213D214C215D216D217A216B3B31A
:10555900500890005BE0655F60028044A229302B0F
:1055690001B340028030A201B35006A200B3B34098
:10557900028023123A8C123ADD9000FCE0B4011348
:10558900A202B34008E5B54440F5B58006E5B55437
:10559900BFF5B575A700D213D214D215C216D2170A
:1055A900A217B3B3500890005CE0655F60028044C5
:1055B900A22A302B01B340028030A201B35006A2C7
:1055C90000B3B340028023123A8C123AE89000FCEF
:1055D900E0B40113A202B34008E5B54440F5B58033
:1055E90006E5B554BFF5B575A700D213D214D21587
:1055F900D216C217E57190689FF8282873025CF8E3
:045609009000D1E05C
:06689F0002560602560934
:10560D009068D2F8282873121EAE8012121EAE803A
:0E561D000D121F388008121FE48003121FE4D4
:0F68D20002561402561902561E02562302562869
:10562B00757102025CF8122110122227A242B340BC
:10563B00229000C5E0F56D900096E0256DFE900080
:10564B0065E075F01E84FC7F00EE2CF5377410902E
:10565B000066F09007CEE0FEA3E0FF740A12702AFA
:10566B00900016E0FCA3E0FD74098F02FF12701A84
:10567B008D078C038E048A058B06126F189007D248
:10568B00EEF0A3EFF09000ECE0B401087430BE0034
:10569B00059F4002800D74309007D2F8E4F0E8A328
:1056AB00F0801B9007D2E0FEA3E0FF74F0BE000376
:1056BB009F500B74F09007D2F8E4F0E8A3F0E537B5
:1056CB0070037537019007D2E0FEA3E0FFE5372F9B
:1056DB00FF50010E9007D2EEF0A3EFF0757103901F
:0356EB000067E075
:0368A50002563167
:1056EE009068E1F8282873802BA243400375710A55
:1056FE008022A243400375710B8019A243400375AB
:10570E00710C8010A243400375710D8007A24340B7
:04571E000375710E90
:1068E1000256F50256F702570002570902571202E3
:0268F100571B33
:10572200025CF89006DDE060031224EA90011CE0BE
:10573200B4011490011DE0A853B800049554500719
:10574200E560C39561400280097415900066F0021D
:1057520057D59000D1E0D39402403F9000A5E024B9
:1057620003A853B80004955450099000A7E0D395BC
:105772006250028008D2017408900066F09000A581
:10578200E0A853B80005D39554500B9000A7E0242D
:1057920003C395625002C20180399000A5E0240340
:1057A200A853B8000495545007E560C395614002C0
:1057B2008008D2017408900066F09000A5E0A8531A
:1057C200B80005D395545009E561240FC395605084
:1057D20002C2019000EBE07007E56BC39414400233
:1057E2008002D201A2014005757104800A75711010
:1057F200900021E4F0A3F0A20BB34029E56875F014
:105802000A84FF7E00900596127051E0C39469509D
:1058120005122407800F9007D0E0F8A3E09007CE8E
:0C582200C8F0A3C8F0025CF89000D1E0D0
:0668A80002572502582AE8
:10582E009068F3F8282873120F108012120F108050
:0E583E000D1210BE800812117080031211703E
:0F68F30002583502583A02583F02584402584999
:10584C009006E1E060031225C6757105025CF81242
:10585C0012B07571069006E5E060031226B690064C
:10586C00E9E06003122792025CF890001AE06006EF
:10587C00A20BB3B34002801D90001AE0252AFFAEA4
:10588C002950010E8E298F2AE55FD394145006906F
:10589C00001AE014F01214F67571079006EDE06032
:1058AC000312286E9006F1E0600312294A025CF89C
:1058BC0090011EE0B40203120E9E1218F5757108C9
:1058CC009006F5E06003122A269006F9E0600312B8
:1058DC002B02025CF8121CB19000DEE0B40305A2AE
:1058EC000BB34002801590001FE0FEA3E0FF740292
:1058FC0012702A90001FEEF0A3EFF0A213B3500524
:10590C00A214B34002800AD213D214D215D216D2EA
:10591C0017757110025CF8025CF8900041E0C394BA
:10592C00465008C2967446900041F090005DE0B479
:10593C00011DE5372406F5379007D2E0FEA3E0FF02
:10594C0074062FFF50010E9007D2EEF0A3EFF090EB
:10595C00005DE0B4021DE537240CF5379007D2E06A
:10596C00FEA3E0FF740C2FFF50010E9007D2EEF057
:10597C00A3EFF085375C755B00900053E0F5741273
:10598C003AF3E55E900041F090000AE55BF0A3E588
:10599C005CF0E574900042F0C2199007D2E0F55B20
:1059AC00A3E0F55C900053E0F574123AF3E55E90D9
:1059BC00003FF0900000E55BF0A3E55CF0E574902F
:1059CC000040F0C218E56EB4010575710B800375CB
:1059DC007103025CF8900045E0C3944650139000AC
:1059EC00ECE0B40104C2968002C295744690004566
:1059FC00F090005EE0B4011DE5372406F537900702
:105A0C00D2E0FEA3E0FF74062FFF50010E9007D2E8
:105A1C00EEF0A3EFF090005EE0B4021DE537240C2D
:105A2C00F5379007D2E0FEA3E0FF740C2FFF500176
:105A3C000E9007D2EEF0A3EFF085375C755B00900B
:105A4C000054E0F574123AF3E55E900045F09000D6
:105A5C000CE55BF0A3E55CF0E574900046F0C21B2E
:105A6C009007D2E0F55BA3E0F55C900054E0F57490
:105A7C00123AF3E55E900043F0900002E55BF0A370
:105A8C00E55CF0E574900044F0C21AE56EB40105D3
:105A9C0075710C8003757103025CF8900049E0C3CA
:105AAC00944650139000ECE0B40104C2968002C2FC
:105ABC00A07446900049F090005FE0B4011DE537FA
:105ACC002406F5379007D2E0FEA3E0FF74062FFF03
:105ADC0050010E9007D2EEF0A3EFF090005FE0B40F
:105AEC00021DE537240CF5379007D2E0FEA3E0FF4A
:105AFC00740C2FFF50010E9007D2EEF0A3EFF0853F
:105B0C00375C755B00900055E0F574123AF3E55E76
:105B1C00900049F090000EE55BF0A3E55CF0E574B5
:105B2C0090004AF0C21D9007D2E0F55BA3E0F55C53
:105B3C00900055E0F574123AF3E55E900047F09052
:105B4C000004E55BF0A3E55CF0E574900048F0C25E
:105B5C001CE56EB4010575710D8003757103025C53
:105B6C00F890004DE0C3944650139000ECE0B40163
:105B7C0004C2968002C297744690004DF09000606B
:105B8C00E0B4011DE5372406F5379007D2E0FEA3FB
:105B9C00E0FF74062FFF50010E9007D2EEF0A3EF3A
:105BAC00F0900060E0B4021DE537240CF537900747
:105BBC00D2E0FEA3E0FF740C2FFF50010E9007D231
:105BCC00EEF0A3EFF085375C755B00900056E0F5C6
:105BDC0074123AF3E55E90004DF0900010E55BF026
:105BEC00A3E55CF0E57490004EF0C21F9007D2E084
:105BFC00F55BA3E0F55C900056E0F574123AF3E522
:105C0C005E90004BF0900006E55BF0A3E55CF0E5E0
:105C1C007490004CF0C21EE56EB4010575710E80D7
:105C2C0003757103025CF8900051E0C39446501365
:105C3C009000ECE0B40104C2968002C2A2744690BB
:105C4C000051F0900061E0B4011DE5372406F537F2
:105C5C009007D2E0FEA3E0FF74062FFF50010E90D8
:105C6C0007D2EEF0A3EFF0900061E0B4021DE5372F
:105C7C00240CF5379007D2E0FEA3E0FF740C2FFF45
:105C8C0050010E9007D2EEF0A3EFF085375C755BF8
:105C9C0000900057E0F574123AF3E55E900051F075
:105CAC00900012E55BF0A3E55CF0E574900052F017
:105CBC00C2219007D2E0F55BA3E0F55C900057E0C1
:105CCC00F574123AF3E55E90004FF0900008E55B36
:105CDC00F0A3E55CF0E574900050F0C220E56EB4E2
:0C5CEC000103756E0075710380028000DA
:1068AE0002585B0258760258BC0258E10259230284
:1068BE0059260259E1025AA7025B6D025C33025C53
:0468CE00F6025CF87A
:105CF80090003FE0B55F028003025D9AA2184072EF
:105D0800900000E0FEA3E0FFEF4E6021AE57AF58D1
:105D1800900000E0FCA3E0FD12000374068E048FDF
:105D280005FF12701A900000ECF0A3EDF09000400F
:105D3800E0601A900000E0FEA3E0FFAC57AD58EF1A
:105D48002DFDEE3CFC900000ECF0A3EDF09000403F
:105D5800E0D39401401A900000E0FEA3E0FFAC57A6
:105D6800AD58EF2DFDEE3CFC900000ECF0A3EDF0FB
:105D7800D218AE55AF56900000E0FCA3E0FDEFC38B
:105D88009DEE9C400D1244CED296C21874C8900065
:105D98003FF0A218B3B3500790003FE0B55F028010
:105DA8000D1244CED29674C890003FF0C2189000ED
:105DB80041E0B55F028003025E55A219407290006F
:105DC8000AE0FEA3E0FFEF4E6021AE57AF58900007
:105DD8000AE0FCA3E0FD12000374068E048F05FFA1
:105DE80012701A90000AECF0A3EDF0900042E06007
:105DF8001A90000AE0FEA3E0FFAC57AD58EF2DFD66
:105E0800EE3CFC90000AECF0A3EDF0900042E0D3E9
:105E18009401401A90000AE0FEA3E0FFAC57AD5889
:105E2800EF2DFDEE3CFC90000AECF0A3EDF0D2194A
:105E3800AE55AF5690000AE0FCA3E0FDEFC39DEE1F
:105E48009C400AC2967446900041F0C219A219B348
:105E5800B35007900041E0B55F02800AC2967446CD
:105E6800900041F0C219900043E0B55F0280030240
:105E78005F1BA21A4072900002E0FEA3E0FFEF4E03
:105E88006021AE57AF58900002E0FCA3E0FD12007D
:105E98000374068E048F05FF12701A900002ECF04E
:105EA800A3EDF0900044E0601A900002E0FEA3E049
:105EB800FFAC57AD58EF2DFDEE3CFC900002ECF026
:105EC800A3EDF0900044E0D39401401A900002E062
:105ED800FEA3E0FFAC57AD58EF2DFDEE3CFC900063
:105EE80002ECF0A3EDF0D21AAE55AF56900002E0E6
:105EF800FCA3E0FDEFC39DEE9C40181244CE900039
:105F0800ECE0B40104D2968002D295C21A74C8900B
:105F18000043F0A21AB3B35007900043E0B55F0204
:105F280080181244CE9000ECE0B40104D2968002AE
:105F3800D29574C8900043F0C21A900045E0B55F4E
:105F4800028003025FECA21B407290000CE0FEA3EB
:105F5800E0FFEF4E6021AE57AF5890000CE0FCA375
:105F6800E0FD12000374068E048F05FF12701A906C
:105F7800000CECF0A3EDF0900046E0601A90000CE5
:105F8800E0FEA3E0FFAC57AD58EF2DFDEE3CFC90D2
:105F9800000CECF0A3EDF0900046E0D39401401A19
:105FA80090000CE0FEA3E0FFAC57AD58EF2DFDEEDE
:105FB8003CFC90000CECF0A3EDF0D21BAE55AF56B4
:105FC80090000CE0FCA3E0FDEFC39DEE9C40159013
:105FD80000ECE0B40104C2968002C29574469000B9
:105FE80045F0C21BA21BB3B35007900045E0B55F54
:105FF8000280159000ECE0B40104C2968002C295BC
:106008007446900045F0C21B900047E0B55F0280DF
:10601800030260BDA21C4072900004E0FEA3E0FFF2
:10602800EF4E6021AE57AF58900004E0FCA3E0FDAE
:1060380012000374068E048F05FF12701A90000474
:10604800ECF0A3EDF0900048E0601A900004E0FE48
:10605800A3E0FFAC57AD58EF2DFDEE3CFC900004DB
:10606800ECF0A3EDF0900048E0D39401401A9000C2
:1060780004E0FEA3E0FFAC57AD58EF2DFDEE3CFC6D
:10608800900004ECF0A3EDF0D21CAE55AF56900092
:1060980004E0FCA3E0FDEFC39DEE9C40181244CE43
:1060A8009000ECE0B40104D2968002D2A0C21C7425
:1060B800C8900047F0A21CB3B35007900047E0B562
:1060C8005F0280181244CE9000ECE0B40104D2962E
:1060D8008002D2A074C8900047F0C21C900049E02A
:1060E800B55F02800302618EA21D407290000EE02F
:1060F800FEA3E0FFEF4E6021AE57AF5890000EE0D0
:10610800FCA3E0FD12000374068E048F05FF1270D5
:106118001A90000EECF0A3EDF090004AE0601A909F
:10612800000EE0FEA3E0FFAC57AD58EF2DFDEE3CAE
:10613800FC90000EECF0A3EDF090004AE0D394013F
:10614800401A90000EE0FEA3E0FFAC57AD58EF2DCB
:10615800FDEE3CFC90000EECF0A3EDF0D21DAE5528
:10616800AF5690000EE0FCA3E0FDEFC39DEE9C400F
:10617800159000ECE0B40104C2968002C2A07446F7
:10618800900049F0C21DA21DB3B35007900049E02A
:10619800B55F0280159000ECE0B40104C29680025D
:1061A800C2A07446900049F0C21D90004BE0B55F54
:1061B80002800302625FA21E4072900006E0FEA306
:1061C800E0FFEF4E6021AE57AF58900006E0FCA309
:1061D800E0FD12000374068E048F05FF12701A90FA
:1061E8000006ECF0A3EDF090004CE0601A90000679
:1061F800E0FEA3E0FFAC57AD58EF2DFDEE3CFC9060
:106208000006ECF0A3EDF090004CE0D39401401AA6
:10621800900006E0FEA3E0FFAC57AD58EF2DFDEE71
:106228003CFC900006ECF0A3EDF0D21EAE55AF5644
:10623800900006E0FCA3E0FDEFC39DEE9C40181221
:1062480044CE9000ECE0B40104D2968002D297C20A
:106258001E74C890004BF0A21EB3B3500790004BB9
:10626800E0B55F0280181244CE9000ECE0B401045F
:10627800D2968002D29774C890004BF0C21E90004C
:106288004DE0B55F028003026330A21F40729000A8
:1062980010E0FEA3E0FFEF4E6021AE57AF5890002C
:1062A80010E0FCA3E0FD12000374068E048F05FFC6
:1062B80012701A900010ECF0A3EDF090004EE06020
:1062C8001A900010E0FEA3E0FFAC57AD58EF2DFD8B
:1062D800EE3CFC900010ECF0A3EDF090004EE0D303
:1062E8009401401A900010E0FEA3E0FFAC57AD58AF
:1062F800EF2DFDEE3CFC900010ECF0A3EDF0D21F6A
:10630800AE55AF56900010E0FCA3E0FDEFC39DEE44
:106318009C40159000ECE0B40104C2968002C2973C
:10632800744690004DF0C21FA21FB3B350079000EF
:106338004DE0B55F0280159000ECE0B40104C29610
:106348008002C297744690004DF0C21F90004FE043
:10635800B55F028003026401A2204072900008E049
:10636800FEA3E0FFEF4E6021AE57AF58900008E063
:10637800FCA3E0FD12000374068E048F05FF127063
:106388001A900008ECF0A3EDF0900050E0601A902D
:106398000008E0FEA3E0FFAC57AD58EF2DFDEE3C42
:1063A800FC900008ECF0A3EDF0900050E0D39401CD
:1063B800401A900008E0FEA3E0FFAC57AD58EF2D5F
:1063C800FDEE3CFC900008ECF0A3EDF0D220AE55B9
:1063D800AF56900008E0FCA3E0FDEFC39DEE9C40A3
:1063E800181244CE9000ECE0B40104D2968002D298
:1063F800A2C22074C890004FF0A220B3B3500790F7
:10640800004FE0B55F0280181244CE9000ECE0B473
:106418000104D2968002D2A274C890004FF0C22024
:10642800900051E0B55F0280030264D2A22140725D
:10643800900012E0FEA3E0FFEF4E6021AE57AF5888
:10644800900012E0FCA3E0FD12000374068E048F96
:1064580005FF12701A900012ECF0A3EDF0900052B4
:10646800E0601A900012E0FEA3E0FFAC57AD58EFD1
:106478002DFDEE3CFC900012ECF0A3EDF0900052E4
:10648800E0D39401401A900012E0FEA3E0FFAC575D
:10649800AD58EF2DFDEE3CFC900012ECF0A3EDF0B2
:1064A800D221AE55AF56900012E0FCA3E0FDEFC339
:1064B8009DEE9C40159000ECE0B40104C296800269
:1064C800C2A27446900051F0C221A221B3B3500772
:1064D800900051E0B55F0280159000ECE0B4010433
:1064E800C2968002C2A27446900051F0C221900068
:1064F800EEE0B402028003026612900089E0D395B0
:10650800675064900089E0F4042567FE9000F1E08C
:106518008E00F5F0E884FF7E008F74EFC39410506E
:106528000CEF8574F0A4FDACF08D7480037574FFD6
:10653800900089E0D39574400B900089E0C395746E
:10654800F572800375720090010CE0D395724006D5
:1065580090010CE0F57290010DE0C3957250069021
:10656800010DE0F5728071900089E0C39567FE9097
:1065780000F1E08E00F5F0E884FF7E008F74EFC331
:106588009410500CEF8574F0A4FDACF08D7480036A
:106598007574FF85745C755B00900089E0255CFF6D
:1065A800AE5B50010E8E5B8F5C74FFBE0009D39FFB
:1065B8004005855C7280037572FF90010CE0D395ED
:1065C80072400690010CE0F57290010DE0C39572DF
:1065D800500690010DE0F572A20BB3B3500D900078
:1065E8008AE0FE9000F9E0D39E5002800A7407907A
:1065F8000066F0C2A1801375A710E5CDC39572405F
:1066080004C2A18002D2A175A700E570C394095005
:106618000AA2EDB34005C2ED123050AE55AF567424
:1066280010C39F74279E400C900088E0C3945A4082
:1066380003026866A210B340091243397406900039
:1066480066F0A224B34008E5B54404F5B58006E534
:10665800B554FBF5B5A212B3500EE562D39433409E
:1066680007E562C394CC4002804190011EE0B40269
:1066780014120E26900090E075F050A4FFAEF08E34
:106688005D8F5E800F90009AE075F050A4FFAEF029
:106698008E5D8F5EE55E455D6011E5B54401F5B53B
:1066A800742B900087F0124449D212900088E0D3EE
:1066B80094014007E562C3941A40028002C2129016
:1066C80006DDE060031224EAA234300301B3501758
:1066D800A234B34008E5B54408F5B58006E5B554DD
:1066E800F7F5B5A23492039006E1E060031225C6DF
:1066F800A235300401B35017A235B34008E5B544BC
:1067080002F5B58006E5B554FDF5B5A235920490BD
:1067180006E5E060031226B6A236300501B3500F35
:10672800A236B34004D2A18002C2A1A2369205903B
:1067380006E9E06003122792A237300601B3500F32
:10674800A237B34004D2908002C290A2379206903A
:1067580006EDE0600312286EA238300701B3501727
:10676800A238B34008E5B54410F5B58006E5B55440
:10677800EFF5B5A23892079006F1E0600312294AB6
:10678800A239300801B35017A239B34008E5B5441F
:1067980020F5B58006E5B554DFF5B5A23992089025
:1067A80006F5E06003122A26A23A300901B3501711
:1067B800A23AB34008E5B54440F5B58006E5B554BE
:1067C800BFF5B5A23A92099006F9E06003122B02D0
:1067D800A23B300A01B35017A23BB34008E5B544C9
:1067E80080F5B58006E5B5547FF5B5A23B920A90D1
:1067F8000088E0C3945A5010E570B40909900088E5
:10680800E004F0757000803BE570B4090375700012
:10681800755600755500758D00758B00756500906F
:106828000087E0C394415008900087E004F0800698
:106838007441900087F0900087E0B44106E5B554B4
:10684800FEF5B5900088E0D394014007E56BC3944A
:106858004140028009740E900066F0124339024BE1
:01686800949B
:106902000000010001400160018001A001C001E01E
:1069120002000300039603B603D603F40400050045
:106922000512052405360548055A056C057E0590B5
:1069320005A805C005DE0600061406280646066EF2
:1069420006AE05CF00FF013F015F017F019F01BF3E
:1069520001DF01FF02FF039503B503D503F303FF34
:1069620004FF05110523053505470559056B057D0E
:10697200058F05A705BF05CE05F1061306270645B7
:10698200066D06AD06ED05DD0FAA0FA50F9F0F9A46
:106992000F940F8D0F870F800F780F710F680F60A4
:1069A2000F570F4E0F450F3B0F300F250F1A0F0ECB
:1069B2000F020EF50EE80EDB0ECC0EBE0EAE0E9FD3
:1069C2000E8E0E7D0E6C0E5A0E470E340E200E0CDD
:1069D2000DF70DE20DCB0DB50D9D0D850D6D0D5411
:1069E2000D3A0D200D050CE90CCE0CB10C940C7671
:1069F2000C580C3A0C1B0BFB0BDB0BBB0B9A0B79E9
:106A02000B570B350B130AF10ACE0AAB0A870A643D
:106A12000A400A1C09F809D409B0098C096709431C
:106A2200091F08FB08D608B2088E086A0846082320
:106A320007FF07DC07B9079607730751072F070DF2
:106A420006EC06CA06AA068906690649062A060A45
:106A520005EC05CD05B0059205750558053C0520E8
:106A6200050504EA04CF04B5049C048204690451B8
:106A720004390422040B03F403DE03C803B2039DAA
:106A8200038903750361034D033B032803160304C3
:106A920002F202E102D102C002B002A0029102821D
:106AA2000273026502570249023C022F02220216B9
:106AB200020901FD01F201E601DB01D001C601BBC1
:106AC20001B101A7019D0194018B0182017901703D
:106AD2000168016001580150014801410139013248
:106AE200012B0125011E01180111010B010500FFF7
:106AF20000FA0FA60FA00F990F920F8B0F840F7C35
:106B02000F740F6B0F620F580F4E0F430F380F2C7D
:106B12000F1F0F120F050EF70EE80ED80EC80EB794
:106B22000EA50E930E800E6C0E580E420E2C0E15F4
:106B32000DFD0DE40DCB0DB10D950D790D5D0D3FE4
:106B42000D200D010CE10CC00C9E0C7C0C590C3577
:106B52000C100BEA0BC40B9E0B760B4F0B260AFD97
:106B62000AD40AAA0A800A550A2A09FF09D409A8DE
:106B7200097C0950092508F908CD08A10875084AB9
:106B8200081E07F307C8079D07730749072006F782
:106B920006CE06A6067E06570630060A05E405BF9F
:106BA200059B057705540532051004EF04CE04AEAB
:106BB200048F047104530435041903FD03E203C76F
:106BC20003AD0394037B0363034B0334031E0308E7
:106BD20002F302DE02CA02B602A30291027F026D32
:106BE200025C024C023C022C021D020E020001F267
:106BF20001E401D701CA01BE01B101A6019A018FC8
:106C02000185017A01700166015D0153014A01416A
:106C1200013901310129012101190112010B01047C
:106C220000FD00F700F000EA00E400DE00D900D326
:106C320000CE00C900C400BF00BA00B500B100AD6B
:106C420000A800A400A0009C009900950091008E6D
:0C6C5200008A008700840081007E007B27
:10009E007548009007DAE4F0A3F075320075310070
:1000AE00754E00754F00C23FD24074FE9007DCF8CB
:1000BE00E4F0E8A3F074FE9007DEF8E4F0E8A3F0B5
:1000CE0074FE9007E8F0745A9007E9F0745A90079E
:1000DE00EAF0D241C233C243C23E22750B00750A0A
:1000EE0000AE0AAF0BAC08AD09EDC39FEC9E4016F7
:1000FE0074FF12700A75CF01780B740126F6500446
:10010E0018E436F650DB22900062E0B4AA1C900789
:10011E0096E0B43C159007D6E0FEA3E0FFEF4E60EC
:10012E0009741EBE0004D39F5003020243755E0085
:10013E00755D0075F8099007D6E0FEA3E0FF740721
:10014E006F4E6006740E6F4E7006743A900796F0FE
:10015E009007D6E0FEA3E0FF7408BE001ED39F40BA
:10016E001A7E017F089007D6E0FCA3E0FD1DBDFFBF
:10017E00011C1200038E5B8F5C801F9007D6E0FE81
:10018E00A3E0FF740812706E8F048E057E017F0847
:10019E00CDCCCD1200038E5B8F5CAE5DAF5E740C6A
:1001AE00D39F74019E500302023EA2F9B3407EE536
:1001BE005E455D700375A382AE5DAF5E74016F4EDA
:1001CE00700375A300AE5DAF5E74026F4E700D903E
:1001DE0007D7E075F002A4FDACF08DA3AE5DAF5E67
:1001EE0074036F4E700375A300AE5DAF5E7403BEF5
:1001FE0000039F5013AC5BAD5CED2FFFEC3EFE9009
:10020E000092127051E0F5A3AE5DAF5EEFB40B0934
:10021E00EEB40105741412700AAE5DAF5EEFB40B4E
:10022E0007EEB4010375F80D785D12707E0201A819
:10023E00900062E4F022755E00755D0075F809901D
:10024E0007D6E0FEA3E0FF7408BE001ED39F401A3F
:10025E007E017F089007D6E0FCA3E0FD1DBDFF01E7
:10026E001C1200038E5B8F5C801F9007D6E0FEA3EE
:10027E00E0FF740812706E8F048E057E017F08CD2C
:10028E00CCCD1200038E5B8F5CAE5DAF5E7411D36E
:10029E009F74019E5003020374A2F9B3500302032C
:1002AE0071E55E455D700375A3D2AE5DAF5E740100
:1002BE006F4E700375A300AE5DAF5E74026F4E702D
:1002CE000D9007D7E075F002A4FDACF08DA3AE5DE6
:1002DE00AF5E74036F4E700375A300AE5DAF5E74B8
:1002EE00046F4E700375A300AE5DAF5E74056F4E66
:1002FE00700375A300AE5DAF5E74066F4E7003752E
:10030E00A300AE5DAF5E74076F4E700375A300AEB3
:10031E005DAF5E74086F4E700375A300AE5DAF5E89
:10032E007408BE00039F5016AC5BAD5CED2FFFEC66
:10033E003EFE90008D127051E5A3F075A300AE5DE8
:10034E00AF5EEFB41009EEB40105741412700AAE6C
:10035E005DAF5EEFB41007EEB4010375F80D785D76
:10036E0012707E02029722755E00755D0075F809A7
:10037E00AE5DAF5E7417BE0004D39F500302044DF2
:10038E00A2F9B3500302044AE55E455D700375A3FE
:10039E00D2AE5DAF5E74016F4E700375A300AE5D9D
:1003AE00AF5E74026F4E700D9007D7E075F002A429
:1003BE00FDACF08DA3AE5DAF5E74036F4E70037532
:1003CE00A300AE5DAF5E74046F4E700375A300AEF6
:1003DE005DAF5E74056F4E700375A300AE5DAF5ECC
:1003EE0074066F4E700375A300AE5DAF5E74076F3B
:1003FE004E700375A300AE5DAF5E74086F4E700352
:10040E0075A300AE5DAF5E7408BE00039F500C90E6
:10041E000070127051E5A3F075A300AE5DAF5E746F
:10042E00166F4E7005741412700AAE5DAF5E7416C0
:10043E006F4E700375F80D785D12707E02037E228A
:10044E00900062E0B4AB0280030204E8755E0075B2
:10045E005D0075F809AE5DAF5E7412BE007CD39F71
:10046E004078A2F9B34070E55E455D700375A382D6
:10047E00AE5DAF5E74016F4E700375A300AE5DAFDF
:10048E005E74026F4E700D9007D7E075F002A4FDFA
:10049E00ACF08DA3AE5DAF5E74036F4E700375A3AB
:1004AE0000AE5DAF5E7403BE00039F5009900075F1
:1004BE00127051E0F5A3AE5DAF5E74116F4E700514
:1004CE00741412700AAE5DAF5E74116F4E700375C8
:1004DE00F80D785D12707E020463229007E5E4F059
:1004EE0074649007D6F8E4F0E8A3F012037574C8AC
:1004FE009007D6F8E4F0E8A3F074FF900070F07463
:10050E00FF900071F074FF900072F0740090006A1A
:10051E00F074FF900073F07400900075F074019009
:10052E000076F090007CE0B4371A900079E09000ED
:10053E0070F090007AE0900071F090007BE09000F7
:10054E0072F080469007E57401F074659007D6F856
:10055E00E4F0E8A3F012037574C89007D6F8E4F03F
:10056E00E8A3F090007CE0B4371A900079E0900098
:10057E0070F090007AE0900071F090007BE09000B7
:10058E0072F0800674029007E5F09007E6E4F074CE
:10059E00669007D6F8E4F0E8A3F012037574C890DD
:1005AE0007D6F8E4F0E8A3F090007BE0B4371290A1
:1005BE000079E090006AF090007AE0900073F0808D
:1005CE00769007E67401F074679007D6F8E4F0E8C9
:1005DE00A3F012037574C89007D6F8E4F0E8A3F000
:1005EE0090007BE0B43712900079E090006AF090B2
:1005FE00007AE0900073F0803E74029007E6F0748B
:10060E00689007D6F8E4F0E8A3F012037574C8906A
:10061E0007D6F8E4F0E8A3F090007BE0B437129030
:10062E000079E090006AF090007AE0900073F0801C
:10063E000674039007E6F022E54F64046006E59920
:10064E0064FF60028031A23F4004D23F8027E54F15
:10065E00600874E6254F900066F0E54E600874F071
:10066E00254E900066F0E54FB4010280FE754F00F6
:10067E00754E00C23F8002C23FE54F90384AF828BF
:10068E002873754F00E599B4FF03754E01E599B4D3
:10069E00FE03754E02E599B4FD03754E03E599B45C
:1006AE00FC03754E04E599B4FA03754E05E599B44D
:1006BE00FB06754F01124339E599B4F906754F04DF
:1006CE00124339E599D394E54007E599C394F04078
:1006DE00028016859950754F027E017F00E550C34A
:1006EE0094E612702A8E338F349007DAE4F0A3F07A
:1006FE00E599D394C44007E599C394E64002802857
:10070E00859950754F0374E5C39550F534753300D4
:10071E00AE33AF34906902126FF9E493F87401931B
:10072E009007DAC8F0A3C8F0D299020C569000795F
:10073E00E07005A231B3400280429007DAE0FEA3DA
:10074E00E0FF74FFBE00039F5009EFC39446EE9482
:10075E000640119007DAE0FEA3E0FFEFD3946DEEB2
:10076E00940640139007DAE0FEA3E0FF9000961285
:10077E007051E599F0800385997580119007DAE044
:10078E00FEA3E0FF900096127051E599F09007DA03
:10079E001270389007DAE0FEA3E0FFEFB40106EE28
:1007AE00B4070280030209FD900796E0B43C028074
:1007BE00030209FDA23150030208E8C29C900079A1
:1007CE00E0900134F090007AE09000A3F090007B6E
:1007DE00E09000C3F090007CE09000ECF090007D83
:1007EE00E0900098F090007EE09000DEF090007FA8
:1007FE00E09000FCF0900080E09000D0F09000813E
:10080E00E09000EEF0900082E090011EF0900083E8
:10081E00E0900182F0900084E0900183F0900085DA
:10082E00E0900184F0123B8A90008BE0900105F07D
:10083E0090008CE09000BCF090008DE09000BDF038
:10084E0074639007D6F8E4F0E8A3F074AB900062FE
:10085E00F012044E900062E4F07464F5097508001D
:10086E001200E9A2234039757401E574D394075040
:10087E002DE5749007D6F8E4F0E8A3F074AA900082
:10088E0062F0120115E574C39407500A7464F509F9
:10089E007508001200E97874740126F650CC803782
:1008AE00757408E574D3940E502DE5749007D6F840
:1008BE00E4F0E8A3F074AA900062F0120115E5745A
:1008CE00C3940E500A7464F5097508001200E97895
:1008DE0074740126F650CC0209E7C29C900134E0F4
:1008EE00900079F09000A3E090007AF09000C3E0C1
:1008FE0090007BF09000ECE090007CF0900098E08F
:10090E0090007DF09000DEE090007EF09000FCE024
:10091E0090007FF09000D0E0900080F09000EEE02C
:10092E00900081F090011EE0900082F07400900023
:10093E0083F07400900084F07400900085F074636E
:10094E009007D6F8E4F0E8A3F074AB900062F012D2
:10095E00044E900062E4F07464F50975080012000C
:10096E00E9757401E574D394075026E5749007D6A3
:10097E00F8E4F0E8A3F074AA900062F01201157486
:10098E0064F5097508001200E97874740126F650B2
:10099E00D3D29C7599FB743C900796F0757408E55C
:1009AE0074D3940E5026E5749007D6F8E4F0E8A3BD
:1009BE00F074AA900062F01201157464F5097508BE
:1009CE00001200E97874740126F650D374C89007AB
:1009DE00D6F8E4F0E8A3F080FE74C89007D6F8E4E9
:1009EE00F0E8A3F0D29C754F00754E007599FB028E
:1009FE000C569007DAE0FEA3E0FFEF4E70068599E5
:100A0E00327531009007DAE0FEA3E0FF74016F4EFD
:100A1E00701BAC31AD32AA33AB34ED2BFBEC3AFA92
:100A2E008A068B07900096127051E599F09007DABE
:100A3E001270389007DAE0FEA3E0FF74026F4E707A
:100A4E0021AC31AD3274566D4C7006E55064E660E3
:100A5E00028003124339123B8A855099754F0075F7
:100A6E004E00020C569007DAE0FEA3E0FF900096CF
:100A7E00127051E599F09007DA1270389007DAE0AB
:100A8E00FEA3E0FFAC33AD348F028E038C068D07D0
:100A9E00906946126FF9E493F9740193FEEAD39EBE
:100AAE00EB994009855099754F00754E00020C5612
:100ABE009007DAE0FEA3E0FF900096127051E599E0
:100ACE00F09007DA1270389007DAE0FEA3E0FFEF3D
:100ADE00B40006EEB401028003020C56900072E0E0
:100AEE00D394C7400B900072E0C394C8F551801A9E
:100AFE00900072E0D39463400B900072E0C3946454
:100B0E00F5518006900072E0F551E55175F002A4A2
:100B1E00FFAEF08F74EF90009612705CEFFCE0FD6C
:100B2E00EC90009912705CEDFCE0FDEC2DB55102DD
:100B3E008003020C470FEF90009612705CE574FF75
:100B4E00E0FCEF90009A12705CECFFE0FCEFC39CAF
:100B5E00B551028003020C47E57490009812705C48
:100B6E00E574FFE0FCEF90009B12705CECFFE0FC84
:100B7E00EF2CB551028003020C47E57490009C12D5
:100B8E00705CE0C39551900079F0E57490009D1271
:100B9E00705CE0C3955190007AF0E57490009E125F
:100BAE00705CE0C3955190007BF0740090007CF077
:100BBE0074FF90007DF0E5749000A012705CE0C3AD
:100BCE00955190007EF0E5749000A112705CE0C328
:100BDE00955190007FF0E5749000A212705CE0C316
:100BEE009551900080F0E57490009F12705CE0C308
:100BFE0095519007D6F8E4F0E8A3F074AB9000623C
:100C0E00F012044E7464F5097508001200E990079D
:100C1E00D612703812044E7464F50975080012006D
:100C2E00E99007D612703812044E7599F97464F56E
:100C3E00097508001200E980FE7599FF7464F509C4
:080C4E007508001200E980FEA8
:0F384A0002069002073B020A00020A73020ABE3E
:100C560022E54E903859F8282873020D699007DA74
:100C6600E0FEA3E0FF900068127051E0F59990074E
:100C7600DA1270389007DAE0FEA3E0FF74116F4EC7
:100C86007003754E00020D69856F99020D69900714
:100C9600DAE0FEA3E0FF900096127051E0F599EFBE
:100CA600B40107EEB40703754E009007DA127038E8
:070CB600020D699007DBE06D
:0F385900020C60020C63020C8E020C94020CB97C
:100CBD00903A0CF8282873855499020D5E85609939
:100CCD00020D5E856299020D5E856699020D5E8547
:100CDD006899807D8569998078856A998073856B1F
:100CED0099806E900022E0F5998066A240B340078E
:100CFD007599FAC2408041A230B3400575990F80B5
:100D0D00359007E5E0600A9007E5E024DCF5998071
:100D1D00169007E6E0600A9007E6E024DEF599807C
:100D2D0006900066E0F599900066E4F09007E5E422
:100D3D00F09007E6E4F0C2308017856C998012853B
:100D4D006799800D856D9980087599FC8003754EA6
:010D5D000095
:103A0C00020CC4020CCA020CD0020CD6020CDC0252
:103A1C000CE1020CE6020CEB020CF0020CF8020DAD
:0D3A2C0047020D4C020D51020D56020D5BBC
:0B0D5E009007DA1270388003123A3957
:03386800020D66E8
:100D690022E538255CFFAE5B50010E9000961270AB
:100D790051E0F539E538255CFFAE5B50010E0FBF38
:100D890000010E900096127051E0F53A85403CE55D
:100D990039B53A058539388041E53AD39539401D49
:100DA900E53AC39539853BF0A4FFAEF0E53C8E04E6
:100DB9008F05FF12701AED2539F538801DE539C305
:100DC900953A853BF0A4FFAEF0E53C8E048F05FF14
:100DD90012701AEDF4042539F53822E53AD395391C
:100DE900401DE53AC39539853BF0A4FFAEF0E53CDB
:100DF9008E048F05FF12701AED2539F538801DE52F
:100E090039C3953A853BF0A4FFAEF0E53C8E048FDB
:100E190005FF12701AEDF4042539F5382290009C6B
:100E2900E0B40170E56875F00A84FF7E008F38E54B
:100E39006875F00A84ADF07C008D3B75400A755BDE
:100E490005755C24E538C394115005120D6A8006B6
:100E59009005CBE0F538E538900090F0E56875F03D
:100E69000A84FF7E008F38E56875F00A84ADF07C4E
:100E7900008D3B75400A755B05755C5AE538C3946E
:100E8900115005120D6A8006900601E0F538E53823
:100E990090001AF02290009CE0B4016AE56875F0B0
:100EA9000A84FF7E008F38E56875F00A84ADF07C0E
:100EB900008D3B75400A755B05755C36E538C39452
:100EC900115005120D6A80069005DDE0F538853868
:100ED9004CE56875F00A84FF7E008F38E56875F087
:100EE9000A84ADF07C008D3B75400A755B05755C25
:100EF90048E538C394115005120D6A80069005EF34
:100F0900E0F53885384D22E56075F00484FF7E00F0
:100F19008F38E56075F00484ADF07C008D3B754039
:100F290004755B01755C00E538C3943F5005120DEB
:100F39006A80069001D5E0F53885382A7529009030
:100F49000065E075F020A4FFAEF09000E7E08E04A4
:100F59008F05FF12701A8D389000CFE0D39560503D
:100F6900030210169000F3E0D395604010ED900154
:100F7900D612705CE0F52C752B000210139000BEA0
:100F8900E0D395604043E5389001D612705CE0F5F6
:100F990039E5389001F612705CE0F53A9000F3E01B
:100FA900F4042560F53B9000BEE0FE9000F3E0F408
:100FB900042EF53CE539B53A058539388003120D1B
:100FC900E485382C752B008041E5389001F61270C4
:100FD9005CE0F539E53890021612705CE0F53A905C
:100FE90000BEE0F4042560F53B9000CFE0FE9000E0
:100FF900BEE0F4042EF53CE539B53A05853938806B
:1010090003120DE485382C752B000210BD9000F6F3
:10101900E0D395605011E53890025612705CE0F506
:101029002C752B000210BD9000BFE0D39560504392
:10103900E53890023612705CE0F539E538900256D1
:1010490012705CE0F53A9000BFE0F4042560F53BCE
:101059009000F6E0FE9000BFE0F4042EF53CE5397F
:10106900B53A058539388003120DE485382C752B7E
:10107900008041E53890021612705CE0F539E538D8
:1010890090023612705CE0F53A9000CFE0F4042546
:1010990060F53B9000BFE0FE9000CFE0F4042EF530
:1010A9003CE539B53A058539388003120DE48538B0
:1010B9002C752B0022900107E0F53D754011755BF9
:1010C90002755C00AE53AF54E53D75F00FA4FDAC5D
:1010D900F0EDD39FEC9E4021E53D8E048F05FF1274
:1010E900701AED75F010A4FFAEF0E56075F011848B
:1010F900FD7C00ED2FF53E800EE56075F01184FF53
:101109007E00EF24F0F53E853E38E56075F01184E8
:10111900AFF07E008F3B120D6A85383FAE53AF5456
:10112900900107E075F00FA4FDACF0EDD39FEC9EA4
:101139004028755B02755C10853E38120D6A853F43
:101149003985383AAE53AF54E53D8E048F05FF1209
:1011590070458D3B853D3C120DE485382A75290083
:10116900752C64752B0022900107E0F53D7540113F
:10117900755B02755C00AE53AF54E53D75F00FA485
:10118900FDACF0EDD39FEC9E4021E53D8E048F052B
:10119900FF12701AED75F010A4FFAEF0E56275F05C
:1011A9001184FD7C00ED2FF53E800EE56275F0118E
:1011B90084FF7E00EF24F0F53E853E38E56275F048
:1011C9001184AFF07E008F3B120D6A85383FAE5314
:1011D900AF54900107E075F00FA4FDACF0EDD39F7B
:1011E900EC9E4028755B02755C10853E38120D6ACD
:1011F900853F3985383AAE53AF54E53D8E048F05A6
:10120900FF1270458D3B853D3C120DE485382A75EA
:101219002900E56C6017E56CC394FE50109000FB43
:10122900E0B402099000E9E0D3940B50028017AEB4
:1012390029AF2AE56C12702A74E78E048F05FF1214
:10124900701A8C298D2A9000D1E0B40453E5607599
:10125900F00484FF7E008F38E56075F00484ADF0FA
:101269007C008D3B754004755B01755C00E538C3F6
:10127900943F5005120D6A80069001D5E0F538AE0D
:1012890029AF2AE53812702A74648E048F05FF127B
:10129900701AAE29AF2AEF2DFDEE3CFC8C298D2A60
:1012A900752C64752B002290009CE0B40146E5681A
:1012B90075F00A84FF7E008F38E56875F00A84AD01
:1012C900F07C008D3B75400A755B05755C00E5385F
:1012D900C394115005120D6A80069005A7E0F538F0
:1012E900AE2BAF2CE5382FFF50010E746412706ECF
:1012F9008E2B8F2C90009DE0B40146E56975F00AAC
:1013090084FF7E008F38E56975F00A84ADF07C00B2
:101319008D3B75400A755B05755C6CE538C39411A6
:101329005005120D6A8006900613E0F538AE2BAF12
:101339002CE5382FFF50010E746412706E8E2B8FBE
:101349002C9000ACE0B40249E56BC3944175F005FB
:1013590084FF7E008F38E56B75F00584ADF07C0065
:101369008D3B754005755B06755C00E538C39413C4
:101379005005120D6A80069006A9E0F538AE2BAF2C
:101389002CE5382FFF50010E746412706E8E2B8F6E
:101399002C9000EEE0B40202800302144FE5607560
:1013A900F01584FF7E008F38E56075F01584ADF087
:1013B9007C008D3B754015755B03755CF4E538C39E
:1013C900940B5005120D6A8006900495E0F538E5F6
:1013D9003875F0FFA4FFAEF09000EFE08E048F05A2
:1013E900FF12701AED900089F0E56775F078A4FF97
:1013F900AEF074FF8E048F05FF12701A8C5B8D5C42
:1014090074028C068D071200398F38AC5BAD5C74A1
:1014190004FF1270458D3B754004755B06755C28A9
:10142900E538C3941D5005120D6A80069006DBE06D
:10143900F538AE2BAF2CE5382FFF50010E7464122E
:10144900706E8E2B8F2C90009BE0B4025DE5627567
:10145900F064A4FFAEF074081200398E5D8F5E74DB
:10146900058E048F05FF12701A8D38AE5DAF5E745C
:10147900058E048F05FF1270458D3B754005755B20
:1014890005755CDEE538C394135005120D6A8006B4
:10149900900687E0F538AE2BAF2CE5382FFF5001C9
:1014A9000E746412706E8E2B8F2C9000DDE0703CF0
:1014B900900065E075F00584FF7E008F3890006527
:1014C900E075F00584ADF07C008D3B754005755BDA
:1014D90005755CC0E538C3941D5005120D6A800678
:1014E900900673E0F538E538900091F0229000A459
:1014F900E0B401179007E1E0252CFFAE2B50010E57
:101509009000F8E012706E8E2B8F2C90011CE0B4C5
:10151900011490011DE0A853B8000495545007E543
:1015290060C39561400280129000C6E0252CFFAE91
:101539002B50010E8E2B8F2C802F9000A4E0B4032A
:1015490016A233B3B350109007E4E0C39405A8532F
:10155900B800069554400280109000C6E0252CFF83
:10156900AE2B50010E8E2B8F2C90009EE0B4020200
:1015790080030218F49000A1E0602FE568D3944637
:10158900402890001BE0FEA3E0FF9000DCE075F02E
:1015990003A4FDACF0EFD39DEE9C400E900100E05A
:1015A900A853B80005D3955450030218F49000D1FC
:1015B900E0B40302800302175885625C755B0090F2
:1015C90000A8E0A853B800049554500E9000A9E073
:1015D900A85BB80005D3955C5003021755E5627501
:1015E900F002A4FFAEF074158E048F05FF12701A75
:1015F9008C068D07900626127051FEE0FFEE9000D2
:10160900A0E0FEEF8E0088F0A4FFAEF074648E04B3
:101619008F05FF12701A8C5B8D5C900065E075F088
:1016290018A4FFAEF09000E7E08E048F05FF12705A
:101639001A8C068D0790063E127051AE5BAF5CE0C6
:1016490012702A74648E048F05FF12701A8C5B8DD8
:101659005CE566A85BB80077D3955C4072E566C324
:10166900955CFFE4955BFE8E5B8F5C7428BE00037E
:101679009F500C755C28755B00740D900066F0AE88
:101689005BAF5C9000A1E012702A74288E048F056C
:10169900FF12701A8C5B8D5CAE29AF2A740A8E0416
:1016A9008F05FF12701A8D068C07AC5BAD5CCFCE2F
:1016B900CF120003740A8E048F05FF12701A8C5B17
:1016C9008D5CAE29AF2A1270768E298F2A807DE52E
:1016D90066A85BB80004955C5072AE5BAF5CE566CA
:1016E90012706E8E5B8F5C7428BE00039F500C7560
:1016F9005C28755B00740D900066F0AE5BAF5C9082
:1017090000A1E012702A74288E048F05FF12701A46
:101719008C5B8D5CAE29AF2A740A8E048F05FF128B
:10172900701A8D068C07AC5BAD5CCFCECF1200036F
:10173900740A8E048F05FF12701A8C5B8D5CAE29BA
:10174900AF2AEF2DFDEE3CFC8C298D2A0218F4906E
:1017590000E9E08560F0A4FFAEF0740512702A7408
:10176900071200398E5B8F5C9000A8E0A853B8007F
:1017790004955450129000A9E075F002A4FDACF054
:10178900EFC39DEE9C40030218F4E56075F00B84ED
:10179900FF7E00900626127051FEE0FFEE9000A039
:1017A900E0FEEF8E0088F0A4FFAEF074648E048F23
:1017B90005FF12701A8C5B8D5C900065E075F0185E
:1017C900A4FFAEF09000E7E08E048F05FF12701AB7
:1017D9008C068D0790063E127051AE5BAF5CE0122D
:1017E900702A74648E048F05FF12701A8C5B8D5CED
:1017F900E566A85BB80077D3955C4072E566C3954A
:101809005CFFE4955BFE8E5B8F5C7428BE00039FD2
:10181900500C755C28755B00740D900066F0AE5B2A
:10182900AF5C9000A1E012702A74288E048F05FF26
:1018390012701A8C5B8D5CAE29AF2A740A8E048FE4
:1018490005FF12701A8D068C07AC5BAD5CCFCECF4D
:10185900120003740A8E048F05FF12701A8C5B8DB7
:101869005CAE29AF2A1270768E298F2A807DE566B3
:10187900A85BB80004955C5072AE5BAF5CE566127C
:10188900706E8E5B8F5C7428BE00039F500C755C74
:1018990028755B00740D900066F0AE5BAF5C90003C
:1018A900A1E012702A74288E048F05FF12701A8C19
:1018B9005B8D5CAE29AF2A740A8E048F05FF127006
:1018C9001A8D068C07AC5BAD5CCFCECF12000374CA
:1018D9000A8E048F05FF12701A8C5B8D5CAE29AFDE
:1018E9002AEF2DFDEE3CFC8C298D2A229000FCE08C
:1018F900B4026AE56075F00884FF7E008F38E56000
:1019090075F00884ADF07C008D3B754008755B016E
:10191900755CE0E538C3943F5005120D6A80069066
:101929000295E0F53885382E752D00AE2DAF2EAC19
:101939002BAD2C12000374648E048F05FF12701AEC
:101949008C2D8D2E900099E08C068D0712702A74CB
:10195900648E048F05FF12701A8C2D8D2EAE29AF5F
:101969002AAC2BAD2C12000374648E048F05FF1270
:10197900701A8C298D2A900099E08C068D071270B7
:101989002A74648E048F05FF12701A8C298D2AA27D
:101999000B401DAE53AF547405BE00039F5002D2D5
:1019A9000BE562D394CC4008D2017411900066F023
:1019B9009000FBE0B402089000E9E0640B6002804B
:1019C90035AE29AF2AE56C12702A74E78E048F05AB
:1019D900FF12701A8C298D2A9000FCE0B40217AE10
:1019E9002DAF2EE56C12702A74E78E048F05FF1255
:1019F900701A8C2D8D2E9000BBE05402601B900054
:101A0900B2E0A853B80012D39554400DA20BB3B35A
:101A19005007E562C3949A40028028AE35AF3690EC
:101A290000B0E075F002A4FDACF0EF2DFDEE3CFC3A
:101A390074022DFD50010CE562BC0007D39D4003E3
:101A4900754401856236753500E5447003021B381B
:101A590090010EE0C395445003021B2A90011EE039
:101A6900C394025076E56875F00A84FF7E009005FC
:101A790096127051E0F55C755B00AE5BAF5C90004F
:101A8900B1E012702A74648E048F05FF12701A8CEB
:101A99005D8D5E90010EE004C395448C068D07129E
:101AA900702A90010EE08E048F05FF12701A8C5D6A
:101AB9008D5EAE29AF2AEF2DFDEE3CFC8C298D2AD7
:101AC9009000FCE0B40212AE2DAF2EAA5DAB5EEF22
:101AD9002BFBEE3AFA8A2D8B2E804690010EE004FC
:101AE900C39544854CF0A4FFAEF090010EE08E043E
:101AF9008F05FF12701A8C5D8D5EAE29AF2AEF2D0E
:101B0900FDEE3CFC8C298D2A9000FCE0B40212AE5B
:101B19002DAF2EAA5DAB5EEF2BFBEE3AFA8A2D8B29
:101B29002E054490010EE0C395445003754400907E
:101B390000BBE05401601B9000AFE0A853B800124D
:101B4900D39554400DA20BB3B35007E560C394CCB1
:101B5900400280259000ADE075F003A4FFAEF0E5EA
:101B6900412FFF50010E74032FFF50010EE560BE97
:101B79000007D39F4003754501856041E545700322
:101B8900021C6B90010FE0C395455003021C5D9048
:101B9900011EE0C394025076E56875F00A84FF7E61
:101BA90000900596127051E0F55C755B00AE5BAF75
:101BB9005C9000AEE012702A74648E048F05FF12E7
:101BC900701A8C5D8D5E90010FE004C395458C06FB
:101BD9008D0712702A90010FE08E048F05FF127095
:101BE9001A8C5D8D5EAE29AF2AEF2DFDEE3CFC8C83
:101BF900298D2A9000FCE0B40212AE2DAF2EAA5D09
:101C0900AB5EEF2BFBEE3AFA8A2D8B2E80469001C4
:101C19000FE004C39545854DF0A4FFAEF090010F88
:101C2900E08E048F05FF12701A8C5D8D5EAE29AFB0
:101C39002AEF2DFDEE3CFC8C298D2A9000FCE0B4A6
:101C49000212AE2DAF2EAA5DAB5EEF2BFBEE3AFA78
:101C59008A2D8B2E054590010FE0C39545500375DC
:101C69004500900111E0252AFFAE2950010E8E2969
:101C79008F2A9000C0E0A829B80004952A5009903D
:101C890000C0E0F52A7529009000FCE0B4020D902F
:101C990000C0E0A82DB80006952E400280099000EA
:101CA900C0E0F52E752D00229000FCE0B401028001
:101CB90003021DBCA20BB35003021DBA9000C7E07A
:101CC900B40168AE29AF2AAC53AD54120003743C79
:101CD9008E048F05FF12701A9000D7E0BC00109D8A
:101CE900400D9000D9E0A829B80004952A5002D2E5
:101CF90002AE29AF2AAC53AD54120003743C8E04D2
:101D09008F05FF12701A9000D7E0C3940ABC001522
:101D1900D39D40119000D9E0C39405A829B80005C6
:101D2900D3952A50028002C2028068AE29AF2AAC3C
:101D390053AD5412000374788E048F05FF12701A84
:101D49009000D7E0BC00109D400D9000D9E0A82973
:101D5900B80004952A5004D2028038AE29AF2AACC3
:101D690053AD5412000374788E048F05FF12701A54
:101D79009000D7E0C3940ABC0015D39D4011900090
:101D8900D9E0C39405A829B80005D3952A50028043
:101D990002C202A202B34019AE29AF2A9000D8E0CC
:101DA90012702A74648E048F05FF12701A8C298DA3
:101DB9002A8002C202A200B34006A201B3B35009AD
:101DC900900021E4F0A3F08024AE29AF2A7400D357
:101DD9009F74019E400C900021E529F0A3E52AF0AB
:101DE900800B74FF900021F8E4F0E8A3F09000DE86
:101DF900E0D39402400C9000C9E07006A20BB3B383
:101E09004002801AAE29AF2A740212702A8E298FD5
:101E19002AAE2DAF2E740212702A8E2D8F2E9000AD
:101E2900C7E0B4011AAE29AF2A740212702A8E29AA
:101E39008F2AAE2DAF2E740212702A8E2D8F2EAEE0
:101E490029AF2A745E12702A740A8E048F05FF1254
:101E5900701A8C298D2A9000FCE0B40217AE2DAFC0
:101E69002E745E12702A740A8E048F05FF12701A7E
:101E79008C2D8D2EAE29AF2A7402BE000AD39F4045
:101E890006752A02752900AE2DAF2E7402BE000A0E
:101E9900D39F4006752E02752D0090001FE529F08D
:101EA900A3E52AF022900065E090039612705CE0A9
:101EB900F542754364900065E0FE9000D2E0D39E40
:101EC9004037E56075F00884FF7E008F38E560755E
:101ED900F00884ADF07C008D3B754008755B037597
:101EE9005C96E538C3941F5005120D6A800690046C
:101EF9004BE0F5388538438035E56075F00884FF97
:101F09007E008F38E56075F00884ADF07C008D3B6C
:101F1900754008755B03755CB6E538C3941F5005B9
:101F2900120D6A800690046BE0F5388538432290DB
:101F39000108E0F53D754011755B04755C00AE5311
:101F4900AF54E53D75F00FA4FDACF0EDD39FEC9EC9
:101F59004021E53D8E048F05FF12701AED75F010D2
:101F6900A4FFAEF0E56075F01184FD7C00ED2FF55E
:101F79003E800EE56075F01184FF7E00EF24F0F5D8
:101F89003E853E38E56075F01184AFF07E008F3BE9
:101F9900120D6A85383FAE53AF54900108E075F0D1
:101FA9000FA4FDACF0EDD39FEC9E4028755B047542
:101FB9005C10853E38120D6A853F3985383AAE5333
:101FC900AF54E53D8E048F05FF1270458D3B853D6D
:101FD9003C120DE485384275436422900108E0F50E
:101FE9003D754011755B04755C00AE53AF54E53D1A
:101FF90075F00FA4FDACF0EDD39FEC9E4021E53DBB
:102009008E048F05FF12701AED75F010A4FFAEF063
:10201900E56275F01184FD7C00ED2FF53E800EE53B
:102029006275F01184FF7E00EF24F0F53E853E389D
:10203900E56275F01184AFF07E008F3B120D6A8561
:10204900383FAE53AF54900108E075F00FA4FDACD2
:10205900F0EDD39FEC9E4028755B04755C10853EBE
:1020690038120D6A853F3985383AAE53AF54E53D8C
:102079008E048F05FF1270458D3B853D3C120DE4A2
:102089008538427543649000D1E0B40479900065C5
:10209900E0FE9000D2E0D39E4037E56075F00884F9
:1020A900FF7E008F38E56075F00884ADF07C008D07
:1020B9003B754008755B03755C96E538C3941F5002
:1020C90005120D6A800690044BE0F5388538438087
:1020D90035E56075F00884FF7E008F38E56075F09E
:1020E9000884ADF07C008D3B754008755B03755C19
:1020F900B6E538C3941F5005120D6A800690046B2B
:10210900E0F5388538432290009CE0B4013BE5684E
:1021190075F00A84FF7E008F38E56875F00A84AD92
:10212900F07C008D3B75400A755B05755C12E538DE
:10213900C394115005120D6A80069005B9E0F5386F
:10214900E5432538C39464F54390009DE0B4013B11
:10215900E56975F00A84FF7E008F38E56975F00A34
:1021690084ADF07C008D3B75400A755B05755C7E1E
:10217900E538C394115005120D6A8006900625E0D2
:10218900F538E5432538C39464F543E5422543F51D
:10219900379000A4E0B402109007E0E02537FE90E4
:1021A90000F8E0F4042EF5379000FBE0D3940140E9
:1021B90040E56CC394E7501D74E7C3956CFE900726
:1021C900E2E08E00F5F0E884FF7E008F38E53725E0
:1021D90038F537801CE56CC394E7FE9007E2E08E82
:1021E90000F5F0E884FF7E008F38E537C39538F5B0
:1021F90037A20B4006E5422464F537E537D39464EA
:102209004009E537C39464F53780037537009000BA
:10221900D4E0C3953750069000D4E0F53722D200B8
:1022290090008FE0A853B800049554504190008F56
:10223900E0A853B800049554500375370F90008FE8
:10224900E004A853B800049554500375370A900068
:102259008FE02402A853B80004955450057537053A
:10226900C20090008FE060067409900066F0C243D6
:102279007E017F009000DAE012702A9000E9E08E7A
:10228900048F05FF12701AE560BC0017D39D401337
:102299009000E3E0B40204D2438002C200740A90C1
:1022A9000066F09000DBE0C3956850159000EDE002
:1022B900A853B8000495545002C200740B900066EC
:1022C900F0E568C39464501D900133E0600D9001FE
:1022D90033E0A853B80006955440028008C2007440
:1022E9000B900066F0A200400375370590011CE0D1
:1022F900B4011490011DE0A853B800049554500787
:10230900E560C39561400280089000C5E0F537801B
:102319003A9000A4E0B40306A233B3B34002802B81
:102329009007E4E0C39405A853B800049554500CF1
:102339009000C5E0F537740C900066F09007E4E072
:10234900A853B8000495545002C20085376D900017
:1023590096E02537FE900065E075F01E84FC7F004D
:10236900EE2CF53722900065E075F00584FF7E00BC
:102379008F38900065E075F00584ADF07C008D3BE9
:10238900754005755B03755CD69000E7E01475F040
:102399000584FF7E00E538BE00039F5005120D6AD3
:1023A900800BE53890046C12705CE0F538E53890E4
:1023B90007E3F09007E3E0FE9000D6E0C39E5008E3
:1023C9009000D6E09007E3F022E56875F00A84FFF3
:1023D9007E00900596127051E0F547E547D3946465
:1023E9004010E547C3946475F00F84FF7E008F4762
:1023F90080037547009000B9E02547F54722900012
:10240900D1E0C3940350269007D0E0FEA3E0FF7407
:1024190004120039E56012702A740F8E048F05FFCB
:1024290012701A9007CEECF0A3EDF080249007D03B
:10243900E0FEA3E0FF7404120039E56212702A7409
:102449000F8E048F05FF12701A9007CEECF0A3EDE2
:10245900F09000ACE0B40262E56BC3944175F005FD
:1024690084FF7E008F38E56B75F00584ADF07C0044
:102479008D3B754005755B06755C14E538C394178B
:102489005005120D6A80069006BDE0F5389007CE1A
:10249900E0FEA3E0FF740A8E048F05FF12701AE5AF
:1024A900388C068D0712702A740A8E048F05FF1264
:1024B900701A9007CEECF0A3EDF09007CEE0FEA3E2
:1024C900E0FF9007D4E0FCA3E0FDEDD39FEC9E4034
:1024D9000F9007D4E0F8A3E09007CEC8F0A3C8F0A6
:1024E900229006DDE090386BF8282873804C8554DB
:1024F9007480479000E9E08560F0A4FFAEF07408AD
:102509001200398F748033856274802E85687480D7
:10251900298569748024856A74801F856B74801A83
:10252900856C7480158567748010856674800B8549
:0A2539006D748006900022E0F57436
:10386B000224F50224F70224FC022510022515027E
:10387B00251A02251F02252402252902252E0225A1
:07388B003302253802253D40
:102543009006DEE0FE9006DFE0D39E404B9006DD72
:10255300E0B404189006DFE0C395745002D23490BF
:1025630006DEE0D395744002C234802A9006DEE092
:10257300C3957450099006DFE0D39574500280022E
:10258300D2349006DEE0D3957450099006DFE0C3A1
:1025930095745002C234802A9006DEE0D3957440CD
:1025A300099006DFE0C3957440028002C2349006AE
:1025B300DEE0C3957440099006DFE0D395744002D2
:1025C300D234229006E1E0903892F8282873804CA8
:1025D30085547480479000E9E08560F0A4FFAEF075
:1025E30074081200398F748033856274802E856875
:1025F3007480298569748024856A74801F856B744F
:10260300801A856C74801585677480108566748064
:0C2613000B856D748006900022E0F574C9
:103892000225D10225D30225D80225EC0225F10208
:1038A20025F60225FB02260002260502260A02262A
:0738B2000F02261402261983
:10261F009006E2E0FE9006E3E0D39E405F9006E175
:10262F00E0B404189006E3E0C395745002D23590DD
:10263F0006E2E0D395744002C235803E9006E2E098
:10264F00C3957450099006E3E0D39574500280024D
:10265F00D2359006E2E0D3957450099006E3E0C3BB
:10266F0095745002C2359006E1E0B401099000F56F
:10267F00E0D3956250028002C235802A9006E2E0D4
:10268F00D3957440099006E3E0C39574400280022D
:10269F00C2359006E2E0C3957440099006E3E0D39B
:1026AF0095744002D235229006E5E09038B9F828AB
:1026BF002873804C85547480479000E9E08560F062
:1026CF00A4FFAEF074081200398F748033856274E2
:1026DF00802E85687480298569748024856A74804A
:1026EF001F856B74801A856C7480158567748010D4
:1026FF00856674800B856D748006900022E0F574FA
:1038B9000226C10226C30226C80226DC0226E1022C
:1038C90026E60226EB0226F00226F50226FA022651
:0738D900FF0227040227098A
:10270F009006E6E0FE9006E7E0D39E404B9006E58C
:10271F00E0B404189006E7E0C395745002D23690E7
:10272F0006E6E0D395744002C236802A9006E6E0B2
:10273F00C3957450099006E7E0D395745002800258
:10274F00D2369006E6E0D3957450099006E7E0C3C1
:10275F0095745002C236802A9006E6E0D3957440F5
:10276F00099006E7E0C3957440028002C2369006D6
:10277F00E6E0C3957440099006E7E0D395744002F4
:10278F00D236229006E9E09038E0F8282873804C82
:10279F0085547480479000E9E08560F0A4FFAEF0A7
:1027AF0074081200398F748033856274802E8568A7
:1027BF007480298569748024856A74801F856B7481
:1027CF00801A856C74801585677480108566748097
:0C27DF000B856D748006900022E0F574FC
:1038E00002279D02279F0227A40227B80227BD02B4
:1038F00027C20227C70227CC0227D10227D60227D8
:07390000DB0227E00227E5CE
:1027EB009006EAE0FE9006EBE0D39E404B9006E9A4
:1027FB00E0B404189006EBE0C395745002D2379006
:10280B0006EAE0D395744002C237802A9006EAE0CC
:10281B00C3957450099006EBE0D395745002800277
:10282B00D2379006EAE0D3957450099006EBE0C3DB
:10283B0095745002C237802A9006EAE0D395744013
:10284B00099006EBE0C3957440028002C2379006F4
:10285B00EAE0C3957440099006EBE0D3957440020F
:10286B00D237229006EDE0903907F8282873804C78
:10287B0085547480479000E9E08560F0A4FFAEF0CA
:10288B0074081200398F748033856274802E8568CA
:10289B007480298569748024856A74801F856B74A4
:1028AB00801A856C748015856774801085667480BA
:0C28BB000B856D748006900022E0F5741F
:1039070002287902287B022880022894022899023B
:10391700289E0228A30228A80228AD0228B202285E
:07392700B70228BC0228C111
:1028C7009006EEE0FE9006EFE0D39E404B9006EDBB
:1028D700E0B404189006EFE0C395745002D2389024
:1028E70006EEE0D395744002C238802A9006EEE0E7
:1028F700C3957450099006EFE0D395745002800297
:10290700D2389006EEE0D3957450099006EFE0C3F5
:1029170095745002C238802A9006EEE0D395744031
:10292700099006EFE0C3957440028002C238900612
:10293700EEE0C3957440099006EFE0D3957440022A
:10294700D238229006F1E090392EF8282873804C6F
:1029570085547480479000E9E08560F0A4FFAEF0ED
:1029670074081200398F748033856274802E8568ED
:102977007480298569748024856A74801F856B74C7
:10298700801A856C748015856774801085667480DD
:0C2997000B856D748006900022E0F57442
:10392E0002295502295702295C02297002297502C3
:10393E00297A02297F02298402298902298E0229E5
:07394E009302299802299D54
:1029A3009006F2E0FE9006F3E0D39E404B9006F1D2
:1029B300E0B404189006F3E0C395745002D2399042
:1029C30006F2E0D395744002C239802A9006F2E001
:1029D300C3957450099006F3E0D3957450028002B6
:1029E300D2399006F2E0D3957450099006F3E0C310
:1029F30095745002C239802A9006F2E0D395744050
:102A0300099006F3E0C3957440028002C239900630
:102A1300F2E0C3957440099006F3E0D39574400245
:102A2300D239229006F5E0903955F8282873804C66
:102A330085547480479000E9E08560F0A4FFAEF010
:102A430074081200398F748033856274802E856810
:102A53007480298569748024856A74801F856B74EA
:102A6300801A856C74801585677480108566748000
:0C2A73000B856D748006900022E0F57465
:10395500022A31022A33022A38022A4C022A51024B
:103965002A56022A5B022A60022A65022A6A022A6C
:073975006F022A74022A7997
:102A7F009006F6E0FE9006F7E0D39E404B9006F5E9
:102A8F00E0B404189006F7E0C395745002D23A9060
:102A9F0006F6E0D395744002C23A802A9006F6E01B
:102AAF00C3957450099006F7E0D3957450028002D5
:102ABF00D23A9006F6E0D3957450099006F7E0C32A
:102ACF0095745002C23A802A9006F6E0D39574406E
:102ADF00099006F7E0C3957440028002C23A90064F
:102AEF00F6E0C3957440099006F7E0D39574400261
:102AFF00D23A229006F9E090397CF8282873804C5E
:102B0F0085547480479000E9E08560F0A4FFAEF033
:102B1F0074081200398F748033856274802E856833
:102B2F007480298569748024856A74801F856B740D
:102B3F00801A856C74801585677480108566748023
:0C2B4F000B856D748006900022E0F57488
:10397C00022B0D022B0F022B14022B28022B2D02D3
:10398C002B32022B37022B3C022B41022B46022BF3
:07399C004B022B50022B55DA
:102B5B009006FAE0FE9006FBE0D39E404B9006F900
:102B6B00E0B404189006FBE0C395745002D23B907E
:102B7B0006FAE0D395744002C23B802A9006FAE035
:102B8B00C3957450099006FBE0D3957450028002F4
:102B9B00D23B9006FAE0D3957450099006FBE0C344
:102BAB0095745002C23B802A9006FAE0D39574408C
:102BBB00099006FBE0C3957440028002C23B90066D
:102BCB00FAE0C3957440099006FBE0D3957440027C
:102BDB00D23B229006FDE09039A3F8282873804C55
:102BEB0085547480479000E9E08560F0A4FFAEF057
:102BFB0074081200398F748033856274802E856857
:102C0B007480298569748024856A74801F856B7430
:102C1B00801A856C74801585677480108566748046
:0C2C2B000B856D748006900022E0F574AB
:1039A300022BE9022BEB022BF0022C04022C09025E
:1039B3002C0E022C13022C18022C1D022C22022C7A
:0739C30027022C2C022C311D
:102C37009006FEE0FE9006FFE0D39E404B9006FD17
:102C4700E0B404189006FFE0C395745002D23C909C
:102C570006FEE0D395744002C23C802A9006FEE04F
:102C6700C3957450099006FFE0D395745002800213
:102C7700D23C9006FEE0D3957450099006FFE0C35E
:102C870095745002C23C802A9006FEE0D3957440AA
:102C9700099006FFE0C3957440028002C23C90068B
:102CA700FEE0C3957440099006FFE0D39574400297
:102CB700D23C22900701E09039CAF8282873804C4B
:102CC70085547480479000E9E08560F0A4FFAEF07A
:102CD70074081200398F748033856274802E85687A
:102CE7007480298569748024856A74801F856B7454
:102CF700801A856C7480158567748010856674806A
:0C2D07000B856D748006900022E0F574CE
:1039CA00022CC5022CC7022CCC022CE0022CE502E8
:1039DA002CEA022CEF022CF4022CF9022CFE022D06
:0739EA0003022D08022D0D60
:102D1300900702E0FE900703E0D39E404B9007012B
:102D2300E0B40418900703E0C395745002D23D90B9
:102D33000702E0D395744002C23D802A900702E067
:102D4300C395745009900703E0D395745002800231
:102D5300D23D900702E0D395745009900703E0C376
:102D630095745002C23D802A900702E0D3957440C7
:102D730009900703E0C3957440028002C23D9007A7
:102D830002E0C395744009900703E0D395744002B1
:102D9300D23D22AE2FAF3074F5D39F74019E40080D
:102DA300782F12707E022EB0753001752F00AE534E
:102DB300AF54E547BE000DD39F40099000CBE0D34D
:102DC300954840028023754800E547C39554F57440
:102DD3009000CEE0D395464008E5462574F546803D
:102DE300069000CEE0F546800205489000A7E0D3A8
:102DF3009562401CE560C395614015AE53AF54E541
:102E030047BE00039F50099000CCE0D39549400290
:102E1300806E9007E7E0A853B800049554500375FB
:102E23004B009007E7E0A853B8000BD39554400636
:102E3300E5549007E7F0E54B7041E554C39547F53A
:102E430074E574D3940540037574059000CDE0C315
:102E530095465007E574C3954640028009E546C38D
:102E63009574F54680069000CDE0F5469000CDE0E0
:102E7300D3954640069000CDE0F5467549008002A3
:102E83000549E54B70169000A7E0C39562500DE528
:102E9300472405A853B8000695544002800F9000BC
:102EA300BAE0F546754B0174789007E7F022AE2F30
:102EB300AF3074E9D39F74039E4008782F12707E5D
:102EC30002304F753001752F00754632A23E402AFD
:102ED3007546199000BAE075F002A4FFAEF0E5481C
:102EE300BE0006D39F4002D23E0548754B0374785B
:102EF3009007E7F0754A0002303EAE53AF54E54702
:102F03006F4E700302303EE547BE000DD39F40096C
:102F13009000CBE0D395484002800F754800E54B05
:102F2300C394035003754619800DE547C39554F5C3
:102F330074E5482574F5489000A7E0D39562400EE8
:102F43009007E7E0A853B80007D395544002800CDC
:102F5300054A9000BAE0B54A03754B00E54BB4034C
:102F630006A20BB3B34002800A054AE54AB43C0308
:102F7300754B02E54BB402299007E7E0A853B8006C
:102F83000ED395544009E5549007E7F0754A009035
:102F930000A7E0C395625009754A0074789007E76B
:102FA300F0E54B705A9000A7E0D39562401CE560B2
:102FB300C395614015AE53AF54E547BE00039F5020
:102FC300099000CCE0D3954940028008754900750B
:102FD300464B8028E554C39547F574E574D39405AF
:102FE30040037574059000A7E0D395624008E54956
:102FF3002574F5498006E5492406F549754A00E537
:103003004B70169000A7E0C39562500DE547240569
:10301300A853B80006955440028003754B01E54B55
:10302300B40118754619054A9000BAE0B54A067509
:103033004B02754A0074789007E7F0E54675F00A8D
:10304300A4FFAEF09007D8EEF0A3EFF022E5709066
:1030530039F1F828287390009FE0700302327790CB
:1030630000D5E0B401028003023192900063E0B521
:103073005F02800302318F7E017F00E5BE12702A5A
:10308300E5BD2FFF50010E8E5B8F5C741012702A0A
:1030930090008EE08E048F05FF12701A9007DCEC0F
:1030A300F0A3EDF074FFBC00039D500B74FF900779
:1030B300DCF8E4F0E8A3F0E56C600FE56CC394FE84
:1030C30050089000FBE06402600280649000E9E035
:1030D300B40B1F9007DCE0FEA3E0FF74E712702A35
:1030E300E56C8E048F05FF12701A9007DCECF0A3D9
:1030F300EDF09000E9E0D3940B40089000D1E06438
:10310300046002802B9007DCE0FEA3E0FF9007DE63
:10311300E0FCA3E0FDEFD39DEE9C400D1270769092
:1031230007DCEEF0A3EFF080079007DCE4F0A3F0F8
:1031330090009FE0B4021E9007DCE0FEA3E0FF9046
:1031430007E8E02FFF50010E74011200399007DCED
:10315300EEF0A3EFF09007DCE0FEA3E0FF9007E8BA
:10316300E0BE0008D39F4004D2418002B2419007E1
:10317300DDE09007E8F09000D1E064016006A24131
:10318300B3B3400280069007DDE0F560023275D2EA
:10319300417E017F00E5BE12702AE5BD2FFF50017D
:1031A3000E8E5B8F5C741012702A90008EE08E047A
:1031B3008F05FF12701A9007DCECF0A3EDF0E56CBD
:1031C300600FE56CC394FE50089000FBE06402605E
:1031D3000280649000E9E0B40B1F9007DCE0FEA3DB
:1031E300E0FF74E712702AE56C8E048F05FF1270FE
:1031F3001A9007DCECF0A3EDF09000E9E0D3940B18
:1032030040089000D1E064046002802B9007DCE06A
:10321300FEA3E0FF9007DEE0FCA3E0FDEFD39DEE0D
:103223009C400D1270769007DCEEF0A3EFF0800760
:103233009007DCE4F0A3F090009FE0B4021E900737
:10324300DCE0FEA3E0FF9007E8E02FFF50010E74DF
:10325300011200399007DCEEF0A3EFF09007DDE0F8
:103263009007E8F09000D1E0640160069007DDE08C
:10327300F560800375600090009BE0700675700137
:1032830002305075BB1802384590009BE070030272
:1032930033FD7E017F00E5BE12702AE5BD2FFF508E
:1032A300010E8E5B8F5C9000E1E0B4010F7E0F7F17
:1032B300FFAC5BAD5C1270768E5B8F5C900106E0B9
:1032C300B40245AE5BAF5C90002BE0FCA3E0FDEDE8
:1032D300D39FEC9E400A90002BE55BF0A3E55CF0E6
:1032E300AE5BAF5C90002DE0FCA3E0FDEFD39DEE61
:1032F3009C400A90002DE55BF0A3E55CF0AE5BAF6C
:103303005C74041200398F62900106E0704CAE5B6E
:10331300AF5C90002BE0FCA3E0FDEFD39DEE9C405F
:10332300091270768E5B8F5C8006755C00755B009E
:10333300AE5BAF5C741012702A90008BE08E048F2A
:1033430005FF12701A8C5B8D5C74FFBC0009D39D62
:103353004005855C6280037562FE9000D1E0B40194
:103363000280030233FBA20BB3B3500E9000A5E01F
:10337300A853B80005D39554500280719000E2E041
:103383008562F0A4FFAEF074648E048F05FF1270A3
:103393001A8C5B8D5CE56C6016E56CC394FE500F74
:1033A3009000FBE0B402089000E9E0640B60028047
:1033B30017AE5BAF5C74E712702AE56C8E048F0561
:1033C300FF12701A8C5B8D5CAE5BAF5C9007DCE028
:1033D300FCA3E0FDEDD39FEC9E4005855C60800B74
:1033E300A241B340069007DDE0F560800BA241B334
:1033F30040069007DDE0F560800375620090009E53
:10340300E0700675700202305075BB1902384590A2
:10341300009EE070030234B2E55FD395524003028D
:1034230034B0900029E0FEA3E0FFE56612706E90D1
:103433000029EEF0A3EFF07E017F00E5BE12702AB3
:10344300E5BD2FFF50010E8E5B8F5C90010BE0708A
:1034530013740A12702A74518E048F05FF12701AA6
:103463008D668019AE5BAF5C740A12702A8F048E6E
:10347300057E017F95CDCCCD126F188F66E566D39F
:1034830094644003756664900029E0FEA3E0FFE5C1
:10349300662FFF50010E900029EEF0A3EFF090008D
:1034A300A2E0048E048F05FF12701A8D66800375E7
:1034B30066329000EEE0700675700302305075BB03
:1034C300130238459000EEE0604A7E017F00E5BEBE
:1034D30012702AE5BD2FFF50010E8E5B8F5C7404C2
:1034E3001200398F679000F0E08567F0A4FDACF01F
:1034F3007464FF12701A8D679000EFE08567F0A483
:10350300FFAEF074FF8E048F05FF12701AED90006A
:103513008AF0800375670090009CE0700675700464
:1035230002305075BB1702384590009CE0B401028D
:1035330080030235C07E017F00E5BE12702AE5BD1F
:103543002FFF50010E8E5B8F5C9007E9E0601990AE
:1035530007E9E01490698A12008CE493FC740193E8
:10356300FDEDC39FEC9E400280069007E9E014F056
:103573009007E9E0C394B3501DAE5BAF5C9007E9DD
:10358300E00490698A12008CE493FC740193FDEFCC
:10359300C39DEE9C400280069007E9E004F090078B
:1035A300E9E0FE9000C2E08E0088F0A4FFAEF07464
:1035B300648E048F05FF12701A8D6880037568008E
:1035C30090009DE0700675700502305075BB1602C1
:1035D300384590009DE0B4010280030236697E0104
:1035E3007F00E5BE12702AE5BD2FFF50010E8E5BF2
:1035F3008F5C9007EAE060199007EAE014906AF4A0
:1036030012008CE493FC740193FDEDC39FEC9E4088
:103613000280069007EAE014F09007EAE0C394B34F
:10362300501DAE5BAF5C9007EAE004906AF41200B1
:103633008CE493FC740193FDEFC39DEE9C400280E8
:10364300069007EAE004F09007EAE0FE9000C8E085
:103653008E0088F0A4FFAEF074648E048F05FF1211
:10366300701A8D69800375690075BB1F0238457E2A
:10367300017F00E5BE12702AE5BD2FFF50010E8EBB
:103683005B8F5C740912702A74E68E048F05FF1237
:10369300701A8D6B9000A4E07006757007023050AD
:1036A30075BB150238459000A4E070030237C47E51
:1036B300017F00E5BE12702AE5BD2FFF50010E8E7B
:1036C3005B8F5C74041200398F6A9000A4E0B4012C
:1036D300159000F8E0856AF0A4FFAEF074071200BD
:1036E30039EF9007E1F09000A4E0B402159000F8E0
:1036F300E0856AF0A4FFAEF07407120039EF90077B
:10370300E0F09000A4E0B4030280030237A7900026
:10371300E5E0701CE56AC394195002D233E56AD31D
:1037230094644002C2339000C4E09007E4F08063E5
:103733009000C4E070349000F8E0856AF0A4FFAE16
:10374300F074FF8E048F05FF12701AED9007E4F0FA
:10375300AE53AF54741EBE0006D39F4002D233E56E
:1037630062D394E54002C2338029E56AC3940A50C8
:103773000DAE53AF54741EBE0004D39F500280029B
:10378300D233E562D394E54002C2339000C4E090A3
:1037930007E4F09007E4E0C394055006740590072E
:1037A300E4F0C2429000A4E0B40414E56AC394199F
:1037B3005002D242E56AD394324002C242C23380FD
:1037C30003756A009000FBE07006757008023050C4
:1037D30075BB14806D9000FBE060567E017F00E5B1
:1037E300BE12702AE5BD2FFF50010E8E5B8F5CEF7A
:1037F300D39421EE940E4005756CFF8015AE5BAF3C
:103803005C741012702A74E38E048F05FF12701A11
:103813008D6CE56C75F00BA4FFAEF09000E9E08EC3
:10382300048F05FF12701A9007DEECF0A3EDF08011
:1038330003756C0090009FE0600575BB1A800375EB
:02384300BB18B0
:1039F10002305902328C0234120234C702352C02D1
:0B3A010035D50236720236A90237D814
:053845000570D2EC2229
:09705C002582F582500205832211
:0F008C0025E050020583258250020583F582226C
:106FF900EF2F500205832582F582E5833E2EF58326
:017009002264
:10706E00CFC39FFF50011E22C3EF9DFFEE9CFE2259
:08707E000806B6000218062204
:0D703800A3E004F07006120049E004F0220D
:0E003900048007C3CE13CECF13CFD5E0F6223E
:106F1800BC000FBE0008ED8FF084FFADF022E4FE48
:106F2800FF22BE000DEF60FE54F0606F20E7030201
:106F38006FCEEAC0E0EBC0E078017A0075F001EEB0
:106F480020E710EF25E0FFEE33FE0AC5F023C5F079
:106F580030E7F0EA5407F9096A7A007B0060010813
:106F6800C3EC9E40167004ED9F4010ED9FFDEC9E13
:106F7800FCE5F0CA4ACA03F5F08005E5F003F5F030
:106F8800C3EE13FEEF13FFD9D77908CACBCAD8D0FE
:106F9800EAFEEBFFD0E0FBD0E0FA22EC8FF084FCB5
:106FA800ED54F045F0C48FF084FEEDC454F045F084
:106FB800C48FF084FDEEC4FE54F02DFFEE540F3C58
:106FC800FEADF07C0022790078008FF0EC7E08207E
:106FD800E70DC3CD33CD33C933C9C833C8DEF08418
:106FE80049F9E5F08FF0BE00E6FD7C00E9FFE8FE18
:016FF8002276
:0E702A00F88FF0A4FFE5F0CE88F0A42EFE2231
:10000300EF8DF0A4F9A8F0EF8CF0A428F8EE8DF0B2
:06001300A428FEE9FF2213
:10700A00600D782B027014007830D8FED5E0F82293
:10701A00EEC0E07E00126F18EFFDEEFCD0E0FE221B
:0C704500EEC0E07E00126F18D0E0FE22CA
:03001B0002001EC2
:0300530002005652
:03009B00020071EF
:0300000002706526
:0970650075817675D000024556D4
:0B705100E5822FF582E5833EF58322E7
:0A0049000582D5820215831582227C
:10001E00C0E0C0F0C083C082C0D075D000124503CE
:0B002E00D0D0D082D083D0F0D0E032E0
:10005600C0E0C0F0C083C082C0D075D00012450693
:10006600D0D0D082D083D0F0D0E032C0E0C0F0C093
:1000760083C082C0D075D000124526D0D0D082D0A1
:0600860083D0F0D0E0324F
:00000001FF
